:020000040000fa
:080000001401040000000000df
:020000040000fa
:10020000140104000000000094010400000000003c
:10021000c2010400000000000e0b040000000000fa
:1002200000000400000000000fea20008079220096
:100230000001880000000000050007000c00070016
:10024000442a0200000000000040da000000fe0026
:100250004440a900003522000000e0000300320005
:1002600000002000a00188004440a8000000060013
:1002700000f3260001002000160037006200400055
:10028000e0804800910188009001ba0062004000bf
:10029000e0804800910188009002ba0062004000ae
:1002a000e08048000002eb006028e10005003a0011
:1002b0008301e90007003300038009000059eb00c7
:1002c000040037006128e100010032000082eb00e9
:1002d00005000700910188001001ba000200e0004b
:1002e000e6ff3a00000005009101880080027800d6
:1002f00062004000e08048003559ba008301e900ff
:10030000080032002559ba008301e90005003200d7
:100310000400e000f4ff320015d9ba008301e900bf
:10032000f1ff3a0000000600881f78000204780000
:1003300082000700080040004f047800000006001b
:100340000000fa00881f7800000478003fb9970089
:10035000ea81570080007800401920007e000700e5
:10036000800078000000e000020035000040eb0053
:1003700000f47800010078004f0478000080fa0053
:1003800000000600889fbe0080047800010078000d
:100390000204780089017800110020000f00070096
:1003a00089007800880f5000010032008000eb00c7
:1003b000010078004f04be00000006000000fa00b3
:1003c0004fb99700e8815700a1ad2000201c200004
:1003d000610007000080fa0000000600e487470083
:1003e000889fbe008a9fbe008c9fbe008e1f780033
:1003f00081bf9f00820078008304780000077800a6
:100400000fb997000116b8008c0578000001eb00c9
:100410000c00e00042003200010178008fb9970023
:100420000300e0003e0032000c00e0002e0032002d
:10043000c900900069009000808f500004003900ce
:1004400009007800f90007000000e00026003500f0
:1004500019a8a300060032000b017800a1002000bb
:100460000e00780036010700000578000100370013
:100470000005eb000b0478000a00e00002003200e7
:100480000e0055000004e80069009000c9019000ca
:1004900003005000880f5000020031000005eb00ff
:1004a00000047800080178008e00780003007800ce
:1004b0002200070008074700888555004900900082
:1004c00008004000c00498000a00e0000400320068
:1004d00009007800230107000000e00002003a0054
:1004e0000b00e000d2ff3a0019b8a300020032006e
:1004f000090078001b01070000c0200019006000ff
:100500000200320049009000e00498000b00560001
:100510008fb99700110009000380d800000178000e
:10052000020078004f0778004f06be004f05be005e
:100530004f04be004f00b1000000060080017800ab
:100540000200e00003003200b15978000201e90026
:10055000fdff3a00000006006200fa00889fbe001e
:100560008a9fbe000004be00020578008300780068
:100570006a80570037010700f88f9f0089979f0016
:100580000000eb00909f9f001a80fb008005fb009d
:100590000000ea00cf04de000904780050022000c9
:1005a000808f550001003a000904e9000800e000ce
:1005b0000c0034000f909700080178008a00780042
:1005c000ff8997000300010080979f008080eb0067
:1005d0000000e000900032001f98970008004000e3
:1005e000909f9f000905450050022000808f550014
:1005f000040032000b00e000e3ff3a009f989700f0
:10060000850037000000eb00f0979f00e0979f0007
:10061000d0979f00c0979f00b0979f00a0979f0022
:10062000b09f9f000900370020c4200000805000c8
:100630000000d00081c4200001004000bf98970056
:1006400090807000b19f9f000a05e8009a00fb00af
:1006500020c4200001010700800078000000e000b5
:10066000f1ff3a00a0c2b3009a4f10000e003a000a
:100670003fb897000080e900b0bf9f0010007800ed
:10068000a09f9f000000e00005003d000000ea0080
:10069000a09f9f003f9897000020a000b09f9f0060
:1006a0000a05e80011003700a19f9f000b003700ea
:1006b000af989700f0ff2700808f500006003200af
:1006c0006a09b9001a00fb000200400001fd2f007a
:1006d00001004000a09f9f000a05e8001a00fb00ef
:1006e000e60007000000e000f1ff3a00e0c2b300be
:1006f0009a4f1000030032000080eb00809f9f00a3
:100700001c003700a0c2b300da4f100007003a0007
:100710003fb897000080e900b0bf9f00100078004c
:10072000809f9f000a05e800120037000000eb00e0
:10073000809f9f000b0037008f989700f0ff2700e5
:10074000808f5000060032006a09b9001a00fb00d1
:100750000200400001fd2f0001004000809f9f002b
:100760000a05e8001a00fb00c40007000000e000d2
:10077000f1ff3a009a00fb0020ca2000b7000700f2
:100780008040eb000000e00001003200ba40780039
:10079000817f9f0080c6b30080cf500004003a00e4
:1007a0009acf100002003a00664050000700370060
:1007b0008f789700c0c6b30080cf500005003a0084
:1007c0009acf100003003a0065404000807f9f00f0
:1007d0000a05e800a0fb2f00008447003a4178009a
:1007e00088017800ea80570060f92f000f00400070
:1007f000760107000000e00006003a00880078005b
:1008000060f92f000f004000a20007000000e00088
:100810005dff3d008080eb00010078004f05be00c9
:100820004f04be000080fa0000000600889fbe0052
:1008300000047800c0019000600090008000eb0090
:10084000808f51003b0039001801780020002900fa
:1008500000006100e20f5000090032000200780041
:100860000090a0000200e0000200350000202400fb
:1008700000007100000c78008080eb002d00370034
:100880000100260001006100810f500008003a00bd
:1008900038009000808f5100050039000800780072
:1008a000300007008080eb000000e00021003a00eb
:1008b00000c020001800600017003a00600220000d
:1008c00008004000a8049000808f540012003a00f5
:1008d00000202000260307008000780020049800f4
:1008e0000000e00005003a0029049800490498003f
:1008f0000900e80030049800060037001860a000e6
:10090000400498000020b00030049800410c98008a
:10091000510c98004d0307002800900050049800e7
:10092000380090006004980000002600180c700049
:100930008000eb00010078004f04be0000000600bc
:100940000200e0000500320090cf100004003200e9
:100950000000e8000201e900fbff3a000000eb00a4
:1009600000000600889fbe00000478000000e00040
:100970000f003a006044b8000800d000a1b2200087
:10098000608078000000e00004003200f5ff0700fe
:100990000000e00001003d008084eb000804e80056
:1009a00009007800e70f540028003c00f2ff3700f0
:1009b00010d8a30024003200a00490004000900052
:1009c000808f54000b003100090150003840900026
:1009d0000000fb0089007800050907000000e00026
:1009e000110034008084440048009000808f54003f
:1009f000f5ff390028009000400498009800780026
:100a000000c020000080600002003200a8049000b6
:100a100001003700b804900001e8a300090032008b
:100a20006904980008003700a8009000410498006d
:100a300061049800510c98001890a0000080eb0011
:100a400002003700590c98000000eb004f04be0074
:100a500000000600010878000000060090cf10009a
:100a6000050032001004e00001003a00000005001b
:100a7000d0cf1000fbff3a00000006000003b100d9
:100a8000030035009000b10001003c00100005009b
:100a9000000005000400fa00889fbe008a9fbe0087
:100aa0008c1f780000047800010678007008900020
:100ab000f8009000010050008808900001005000ec
:100ac0009808900001005000a80890000100500014
:100ad000b808900001005000c8089000810550003f
:100ae0000002220090bf9f0000032300a0bf9f00d0
:100af000081090000028a30018003a000b00e00046
:100b0000160034000b0578008a047800e20f5500c7
:100b100001003600290020000900e0000c0034002c
:100b200058009000c801900009017800ee8057003d
:100b300003000100500498008080eb000000e000fa
:100b40009c0032006808900009004000600c98008a
:100b5000090555004240a900ebff3c0078019000d8
:100b60000200e0000c00340058009000c801900022
:100b70008c00780003000100500498008080eb0096
:100b80000000e0008b00320068089000f800900040
:100b900001004000600c9800080890000000e00090
:100ba00016003400000578008a047800e20f550032
:100bb00001003600290020000900e0000c0034008c
:100bc00058009000c801900009017800ec8057009f
:100bd00003000100500498008080eb000000e0005a
:100be000740032006808900009004000600c980012
:100bf000090555004240a900ebff3c001809900090
:100c00000200e0000c003400e80090005800900062
:100c1000c801900003000100500498008080eb00a0
:100c20000000e0006300320068089000980890001f
:100c300001004000600c9800280890000000e000cf
:100c400016003400000578008a047800e20f550091
:100c500001003600290020000900e0000c003400eb
:100c600058009000c801900009017800ec805700fe
:100c700003000100500498008080eb000000e000b9
:100c80004c0032006808900009004000600c980099
:100c9000090555004240a900ebff3c0038099000cf
:100ca0000200e0000e003400e800900018089000f8
:100cb0008080400058009000c801900003000100af
:100cc000500498008080eb000000e0003900320002
:100cd00068089000b808900001004000600c98007f
:100ce000480890000000e00016003400000578007d
:100cf0008a047800e20f5500010036002900200028
:100d00000900e0000c00340058009000c801900079
:100d100009017800ec80570003000100500498009e
:100d20008080eb000000e0002200320068089000a4
:100d300009004000600c9800090555004240a900d8
:100d4000ebff3c00081090000028a30018003200c0
:100d50000b00e000160034000b0578008a047800d0
:100d6000e20f550001003600290020000900e000d4
:100d70000c00340058009000c80190000901780070
:100d8000ee80570003000100500498008080eb00c3
:100d90000000e000070032006808900009004000f1
:100da000600c9800090555004240a900ebff3c008b
:100db0008000eb00010078004f0678004f05be0070
:100dc0004f04be000080fa0000000600889fbe00ad
:100dd0008a1f78000004780001027800024578003c
:100de000830478000200fb00cf80de005002b100d7
:100df0000180b10032052000820f5000e08f5800c2
:100e000095013e00006001008d013700920137001e
:100e100091013700900137008f0137008e013700b4
:100e20008d0137008c0137008b0137008a013700b4
:100e300089013700880137008701370086013700b4
:100e400085013700840137008301370082013700b4
:100e500081013700800137007f0137007e013700b4
:100e60007d0137007c0137007b0137007a013700b4
:100e70007901370078013700ed003700760137003f
:100e80007501370074013700e9003700e8003700ca
:100e9000e7003700700137006f0137006e0137003f
:100ea0006d0137006c0137006b0137006a013700b4
:100eb00069013700680137006701370066013700b4
:100ec0004b013700640137006301370062013700ce
:100ed00061013700800037005f0137005e01370095
:100ee0005d0137005c0137005b0137005a013700b4
:100ef0005901370058013700cd003700560137003f
:100f0000150037001c003700c9003700c800370043
:100f1000c700370050013700170037004e01370077
:100f20004d0137004c0137004b013700ec00370012
:100f3000690037001f0137004701370046013700bd
:100f40002b013700440137006300370042013700ae
:100f500041013700600037006e0144001200780044
:100f6000808141009480e900010a78000009e800ce
:100f70009149780041013700a8609000c0c6b300d5
:100f800080cf50000a003a0094007800648050003e
:100f9000000a78001000be004f89de00cf91de000d
:100fa0000002be00020378008203780015003700bb
:100fb00010c7b30080cf500002003a00140178003f
:100fc0000400370014017800a0c6b30080cf5000a1
:100fd00005003a0068005100000a78003002be00a7
:100fe0002003be00070037000280e900000a7800f5
:100ff0001000780000027800cfa2de000503780020
:1010000086037800049cbe000694be00a860900091
:1010100080c6b30080cf50000f00320020c6b3005e
:1010200080cf500006003a00184078000000fb0016
:10103000cf80de0001017800820178000a003700cd
:1010400040c7b30080cf500003003200664040002c
:1010500080cf500006003a0018007800cf80de00f4
:101060000101780082017800009cbe000294be005d
:101070003800be002801be00e00f5000e08f58008d
:10108000e00f5900e08f590004003d006e0144005c
:1010900092007800d0c2b3000c0037000810900016
:1010a0000018a300040032006e0144009200780092
:1010b000b0c2b300050037000008a300570032009b
:1010c0006e0144009200780000c2b30080f4780002
:1010d0000109e80051003700a8609000c0c6b300c5
:1010e00080cf500006003a009400780064805000e1
:1010f000000a78001002be006033b8001500370007
:1011000010c7b30080cf500002003a0014017800ed
:101110000400370014017800a0c6b30080cf50004f
:1011200005003a0068005100000a78003002be0055
:101130002003be00070037000280e900000a7800a3
:101140001000780000027800050020000600200052
:1011500007002000049cbe000694be00a86090001a
:1011600080c6b30080cf50000f00320020c6b3000d
:1011700080cf500006003a00184078000080fb0045
:101180000100200002002000030020000a003700b8
:1011900040c7b30080cf50000300320066404000db
:1011a00080cf500006003a001800780001002000af
:1011b0000200200003002000009cbe000294be003c
:1011c000081090000038a300140032003800be0060
:1011d0002801be00e00f5000e08f5800e00f5900da
:1011e000e08f59000d00320080c7b300804f5500da
:1011f0000300320080c5b300804f550007003a005d
:101200006e0044009000780002c3b30082f47800be
:101210008100e8008af478000108e8007800900076
:1012200000804400600498008a4078006d00370018
:10123000a860900014017800c0c4b30080cf5000b3
:1012400005003a0068005100000a78005001be0015
:101250004000be000400370064005100000a78001e
:101260001000be00a2080700009cbe000294be0051
:10127000380090000000e00004003d006e014400d2
:1012800092007800d0c2b3000c0037000810900024
:101290000018a300040032006e01440092007800a0
:1012a000b0c2b300050037000008a30005003200fb
:1012b0006e0144009200780000c2b30080f4780010
:1012c0000109e80078009000008044006004980064
:1012d0008a40780008007800d901070067003700cd
:1012e000286090008000fb00c0062000808f500026
:1012f000230032000a003c0064005000808f500040
:101300002600320004003c0066005000808f500030
:101310000b00320021003700a00620000500370036
:1013200040072000808f50001c0032001b003c0052
:1013300063005000808f5000070032001700370014
:101340001480e900000a780010007800485c9000e2
:1013500008487800490037001480e900000a780046
:101360001002780068089000cf80de00010178004c
:1013700082017800009abe000292be003f00370052
:101380001480e900000a78001001780068089000d5
:10139000cf80de000089be00380037001480e900ed
:1013a000000a780010007800680c900008087800a7
:1013b000320037001480e900000a7800100078003d
:1013c000cf80de000101780082017800009cbe0021
:1013d0000294be00780090000080440060049800f1
:1013e00081c7b30008007800dc0007002300370045
:1013f0001480e900000a780010007800600498006a
:10140000580990000200e00002003d00850107003d
:10141000090037008000eb0049fd070080007800dc
:101420000000e000030032006800900000805000df
:101430000100370058089000100c98000f0037008a
:101440006e0144009200780050c2b30080f1780031
:101450000109e80009003700ee004400110078009f
:10146000808144000a4278008008e8000a04e00015
:1014700001003a0054c2b300844978000000eb0038
:101480004f0578004f04be0000000600889fbe0094
:1014900080047800f1628000010078000100e00023
:1014a0000a003a0001c62000600ce2001c00320075
:1014b00011007800908f5400140036008080e800fe
:1014c0001100e000faff3a00150037001100e000bb
:1014d0000600320011017800928f54000b00360094
:1014e0008280e8001100e000faff3a001001780065
:1014f00001c6200000638000820f50000800320007
:1015000011007800908f540002003e000100780026
:10151000150037008080e800910f1100f8ff3a00b5
:1015200018638000890f540001003100090478001d
:101530000800780099030700000178000000e0002f
:1015400005003a000000eb00890f5400060032004d
:101550000804d100f3ff3700081978000200780072
:1015600095030700cbff37004f04be0000000600c4
:10157000881f7800630440000800a1000001eb0010
:10158000800f540022003600e30f540001003e009b
:101590004800200008007800bcff070080007800a9
:1015a0000001eb000000e00019003200100178009b
:1015b0009201780064805100880f500003003100d0
:1015c00012009000800878000700370008004100f2
:1015d0008008780012029000140098001100780032
:1015e0000888510008097800910078000100e000a7
:1015f00004003200110090008180e8000000e0004b
:1016000001003a008000eb00f16288000281e800ee
:10161000020078004f04780000000600881f780060
:10162000880020000800d000a1b22000608078006f
:101630000000e000010032000a0007000804e90091
:10164000f8ff3700e0b0200094033700664ce2005a
:1016500003003a00fbff070020c0b30066ecb700b0
:1016600000000600889fbe0000047800bdfc070053
:10167000800478001868a30002003200280090005f
:101680004d0307000000eb00200498003840900054
:101690000004e000050035000000fb000206070022
:1016a0000000e000010032008084eb001810900080
:1016b0000000e00008003200040607000000e0001f
:1016c000010032008084eb00181090003a030700fc
:1016d0000000eb00101498001878a3000e003200f0
:1016e0008000eb000100d000a2b220000200400008
:1016f000900f1400060032008100e800e78f5000d0
:10170000f8ff3600080078002b03070010003700b0
:101710000008eb00fbff3700000ceb0000c0eb0003
:101720003044980060022000080040002004980027
:101730004004980050049800400c98006004980001
:10174000500c98007004980076004400000c98003b
:10175000090078004f04be00000006006f02b000d0
:10176000889fbe008a9fbe008c9fbe008e1f78009f
:101770008006780010bd2000b0b79f0080c5b30080
:1017800080cf50000200320002bc2000b2b79f00a0
:1017900083002000c3b79f00f0c6b30080cf500085
:1017a0000a0032006940400080cf5000050032003e
:1017b000a4002000c4b79f0080c5b30080cf5000b4
:1017c00002003a0000012000c0b79f008e012000f7
:1017d0003d04be002d05be0040c6b30080cf5000c2
:1017e000030032006540400080cf50000a003a00fc
:1017f000e00f5400e08f5c00e00f5d00e08f5d00c3
:1018000005003d000800be000a01be0057070700a2
:101810000205be000004be00e00f5400e08f5c0033
:10182000e00f5d00e08f5d0003003a005d0890006e
:101830000000e0000c0032007e012000cfb09700d5
:1018400001027800cfa2de0005037800860378004d
:101850000800be000a01be00da0707003fb2970089
:1018600064407800d0e79f004fb09700cf80de0043
:101870000101780082017800d0b79f00e1b79f0096
:10188000f2b79f0083bf9f000203be000002be00ac
:101890000800be000a01be00c3070700809ebe000c
:1018a0008296be00e00f5000e08f5800e00f590014
:1018b000e08f5900220034000e00e00020003400c8
:1018c0003d00be002d01be005fb29700efb2970051
:1018d0007fb397008fbb9700be0707000205be00cd
:1018e0000004be000e07e900e1fc2f008f804000dd
:1018f000010647005fb29700efb297007fb39700f1
:101900008fbb97000800be000a01be004e0807000a
:101910001d0010003fb19700624e7800889ebe0007
:101920008a96be00e00f5400e08f5c00e00f5d007f
:10193000e08f5d00020034000e00e000e0ff3c009c
:10194000cfb19700e88f510010003a000d109000c1
:101950000038a3000d003200f70f570006003e00cc
:10196000e4fc2f000e024200e4c07f0000c3b3007d
:1019700080cf5000050032000e07e90000c3b3001d
:10198000e1fc2f008e80400080f07f00780117007e
:10199000920e98006d009000e3fc2f008f814100b3
:1019a0008e804100e5fa07001d0e90005d08900052
:1019b000800f560006003d000c005000800e98007d
:1019c0000d1090000040a100801698000f00370015
:1019d0000000e0000d003d000d109000740060005c
:1019e000f00f500009003a007d089000fd009000c3
:1019f000010050008d089000010050000c075000bd
:101a00004240a900010034008e0e98004f07780074
:101a10004f06be004f05be004f04be006f02b1006e
:101a200000000600800078001004e0000200320090
:101a30005104e000feff3a00008050000000060064
:101a4000ef04b000889fbe008a9fbe008c9fbe003e
:101a50008e1f7800c0af9f00a1df9f0060fa2f00ab
:101a60000f004000e0af9f00cfaa97005503be00d3
:101a70004502be0084af9f0095af9f00a6af9f00b8
:101a8000b7af9f0010c6b30080cf500016003200e1
:101a900010c4b30080cf5000130032004fab97004a
:101aa000560890000000e00003003d0060002000a8
:101ab000500b98000c0037000000e0000a003a00cc
:101ac00070c6b300afdb970080cf53000300320035
:101ad00070c4b30080cf530003003a001000200010
:101ae000cfa89700d0089800cfa89700e2fc2f005d
:101af000028047007602070080017800e20f500064
:101b000014003a00cfa99700e300900030002000b5
:101b10009009980010c6b3002fda9700804f52004a
:101b20000a00320064404000804f5200070032003b
:101b30000040e800804f52000400320002c720003d
:101b40000040e800804f520017003a0042c72000d2
:101b5000150037000000e00018003400cfaa9700fd
:101b6000e500900030002000900a980010c6b300f5
:101b70002fdb9700804f53000a0032006440400082
:101b8000804f5300070032000040e800804f5300b0
:101b90000400320082c720000040e800804f53005c
:101ba00001003a00c2c72000b25878000200780055
:101bb000b058780090487800f201370014c6b3009e
:101bc000afdb970084cf53000300320010c4b30092
:101bd00080cf530010003a004fa89700ec0040005f
:101be0001101780000c3b300005978008208e800b2
:101bf00080c7b300afd8970084cf500001003200f7
:101c000080c5b300004978004fa99700720090008a
:101c10000080e800700198000300e00003003a0033
:101c20008006eb00fda79f00d001370011c6b3006e
:101c3000afd9970081cf51000300320010c4b30028
:101c400080cf5100ad003a000ec820002fda970077
:101c5000814f5200010032001ec92000cfaa970018
:101c6000550890008006e8000000e00001003d00fb
:101c70001d0220000d06e8004fab97003604be00a1
:101c80002605be006022b8006033b8000fa8970098
:101c90009fa897002fa99700bfa997008f0707005b
:101ca0000000e00001003d000bf0a20088af9f00a3
:101cb00099af9f00aaaf9f00bbaf9f007fa0970086
:101cc00064005000f0a79f00efab9700805beb0033
:101cd000e7af9f003f003700c20120000300200053
:101ce00001fd2f0001804700270207000faa97007f
:101cf0009faa97002fab9700bfab9700f4af9f0050
:101d000085b79f0096b79f00a7b79f000400be004d
:101d10000601be00760707000004be000005be00f5
:101d2000670656004240a9000c0034009c070700db
:101d30000002be000203be007fa897008fb097008c
:101d40001fb19700afb197009807070080af9f00c1
:101d500091af9f00a2af9f00b3af9f00efaa970083
:101d6000e7824200e5af9f0070002000e00f5400c2
:101d7000e08f5c000d003400600020006fab970026
:101d80006f636500e6af9f00cc5bdd004455de006d
:101d90000a857300c4ddde00e00f5500e08f5d00b2
:101da000020034000000e900f4ff3b000000e900fd
:101db00005003300efa897008060eb00e1af9f00c3
:101dc0000000e900fbff3b006fa99700670141009d
:101dd000e2af9f000c00e000090034006022b80070
:101de0006033b8000fa897009fa897002fa997000d
:101df000bfa997006f0707000000e000b6ff3c0096
:101e0000efa9970064fa2f000f02420004805100ee
:101e10000006e90075fa2f0085824700e5af9f00b4
:101e20008d0f560001003d008c0678000d00e0008b
:101e30002b0035008c8f560005003d006fab9700de
:101e400066c07e00f2c0b300e74f500001003c00c6
:101e50000041eb008d00e900efab970067c0780010
:101e6000824f500006003a008d06e9008100e9002b
:101e7000efa9970063c07800824f5000faff32004c
:101e8000ef4f510004003a006faa970064c0780039
:101e90000040e80000f278000100e00007003d008b
:101ea000efaa97008502e900e5af9f008d06e800e4
:101eb0007fa0970064004000f0a79f008d00e9001c
:101ec000070033006fab970066c078000000fb008e
:101ed0006e40780000f378008100e900f9ff3b00d4
:101ee000cfab9700570890000000e0001f013d00b5
:101ef0000d00e900d00b98001c0137000fac9700d3
:101f00009fac97002fad9700bfad97006022b8003f
:101f10006033b8000800be000a01be00ef060700eb
:101f20000000e00005003d000bf0a20088af9f001c
:101f300099af9f00aaaf9f00bbaf9f007fa0970003
:101f4000725927000280b900026a2800130020009d
:101f5000f2040700e4005000f1a79f001d003b00c1
:101f600063801000c1ff2f00010460000800ea0038
:101f7000f0a79f008004eb000800e0004700340059
:101f80000808a3000e0032006848b800a2b3200081
:101f9000020040003002be002003be000fa89700e0
:101fa0009fa897002fa99700bfa9970006070700d1
:101fb00080af9f0091af9f00a2af9f00b3af9f0083
:101fc0000884d1008904e8000800e000ecff3c0030
:101fd000320037000100e000300034006022b80019
:101fe0000600200007ff2300b4b79f00c5b79f007d
:101ff000d6b79f00e7b79f00c0ff2f0000806000aa
:10200000f0a79f00000478008004eb001600340065
:102010000808a300100032006848b800a5b32000eb
:10202000050040003002be002003be003fb0970014
:10203000cfb097005fb19700efb19700e2060700bd
:102040000002be000203be00b4b79f00c5b79f00e8
:10205000d6b79f00e7b79f000884d1008904e80045
:102060000800e000eaff3c003fb29700cfb29700c3
:102070005fb39700efb397000fa897009fa8970052
:102080002fa99700bfa997004407070080af9f00c2
:1020900091af9f00a2af9f00b3af9f004fab9700df
:1020a000d608900060c6b300afdb970080cf530026
:1020b000040032006687400060c4b30080cf530044
:1020c00003003a007fa09700008040006a074000ac
:1020d000f30f5700010034003e01200000c3b3009d
:1020e000efa8970080587800e1af9f003a003700d2
:1020f0000800be000a01be007d0607000006be0003
:10210000f0b79f0081bf9f00680757004240a900b9
:102110000e003400a20607000002be000203be004b
:102120000800be000a01be00a00607006022b80039
:1021300046782d0077192400a306070080af9f0082
:1021400091af9f00a2af9f00b3af9f00efa9970090
:10215000e8814100e3af9f0088002000e00f5600b7
:10216000e08f5e001100340078002000a200200003
:10217000030020007fb097008fb897007801070018
:102180006faa970005c3b30005624100e4af9f004a
:10219000f0b79f0081bf9f00e00f5000e08f580014
:1021a000020034000804e900f0ff3b000804e900e5
:1021b0000600330000c3b300efab970080637800e4
:1021c000e7af9f000804e900faff3b006fa8970003
:1021d00068004000e0af9f000e00e0000b003400fc
:1021e0000fac97009fac97002fad9700bfad970045
:1021f0006022b8006033b8000800be000a01be00cb
:102200006c0607000000e000b9ff3c00efa8970053
:1022100062fa2f000f014100028050000007e90020
:1022200073fa2f0083814700e3af9f007fa09700e0
:1022300067004000f0a79f0001c3b30093cf1000d8
:102240000a003a000e07e9007fa097000000e900ad
:10225000f0a79f006faa97000402e800e4af9f0078
:1022600014427800814f5200f6ff3200cfaa970047
:10227000d508900060c6b3002fdb9700804f530055
:102280000300320060c4b300804f530004003a00e2
:102290007fa09700008040008006e8000a00370019
:1022a0008001eb0050c6b300afdb970080cf530036
:1022b0000300320050c4b30080cf530001003a0045
:1022c00013002000838640008d0f570001003d0061
:1022d0008e0678000d00e000240035008e8f560039
:1022e00006003d006fa89700e0c07e0092c3b300d7
:1022f00040c3b30080cf500001003c0002c3b300d4
:102300008d00e900efa9970063c07800824f50006c
:1023100006003a008d06e9008100e9006faa9700e7
:1023200064c07800824f5000faff320090c3b300bf
:10233000804f510004003a00efaa970065c0780072
:102340000040e80080f278000100e00007003d0056
:102350006fab97000603e900e6af9f008d06e8002b
:102360007fa097000000e800f0a79f007fa29700e1
:102370008d0178006fa99700afd897004fa89700fc
:102380000e0107004f0778004f06be004f05be0044
:102390004f04be00ef04b100000006000000e000a2
:1023a00003003400d2020700e10f400001003a00b0
:1023b0000000eb00000006000000e00036003200e4
:1023c0000081e90012027800e30f5200320036006b
:1023d0000408a30030003a00016380000100e0001f
:1023e00002003200810f5100030031000108780023
:1023f000026388001d003700810178001100900001
:102400000000e00008003200820f5000060031009a
:1024100080017800100090000000e000020032000f
:10242000820f5000faff39009300780001804100cc
:10243000800f510018003900820f500003003a004d
:102440008489400003017800080037009300900061
:102450000100e0000300320004004100808f5000c2
:102460000d0039001101980092019800920090002f
:102470000100e000080032009201780003004100f2
:10248000810f500004003a005e2cef0010894100db
:102490001000900010019800000006000001780074
:1024a000000020000000e000080032000000800072
:1024b0000000e000050032000000e9000000880094
:1024c0000000d0000100800002b07800000006008b
:1024d000889fbe00800478000104780031009000dd
:1024e0000000d0004501de00f07f2000800f510089
:1024f00010003a00800ceb00310090006f0060008b
:1025000008003a00210090000000e00005003a00b9
:10251000110090000000e00002003a001100e0000d
:1025200002003200200020001500370010002000bb
:10253000130037000200e00005003c0001007800b5
:10254000cf010700000178000000e0000a003c0015
:1025500038009000f10028000100600001fe230017
:10256000010070003004980020c02f00800c410052
:102570000080eb0002003700800ceb000000eb0055
:102580004f04be0000000600881f78008a9fbe002e
:10259000000478000205be00300190000200d00067
:1025a000c500de00f07f2000808f50000c003a0054
:1025b0006f00610008003a00280090000000e00071
:1025c00005003a00180090000000e00002003a0008
:1025d0001800e0001c003200200020005d003700e1
:1025e0000100e00006003a0008007800a40107009e
:1025f000800078000000eb000100e00055003c0086
:102600006108b9000a0540008b854800e07f200082
:10261000800f5500e08f5d000d0034003800900001
:102620006022b8000600200007ff2f000000e00035
:10263000030035006022b8000600200007ff2700d5
:10264000049cbe000694be0010002000410037002c
:10265000b8009000e00f5500e08f5d0005003400e9
:10266000f000280000806000c450dd000100700010
:102670003600370000002800808260006f80600014
:102680000040a0003004980061055500e0855d0021
:10269000c0fc2f00f1ff2f00800f5500818f5d00df
:1026a00006003d00350498000000eb00200498006f
:1026b00010049800000ceb00260037000a02780096
:1026c000f00f45000b003c0018009000000c780053
:1026d0002800900010049800380090002004980012
:1026e0000000eb003004980070024200f00f42003e
:1026f000f5ff34000402ea001200320018017800ed
:102700000411de00f0011200180090008300dd00cb
:10271000010c71000400de00280190008310dd0030
:1027200001007000100498000411de0038009000d1
:102730008301dd0003017100220498000400de0023
:1027400030049800380090000500700030049800b4
:102750000080eb004f05be004f047800000006002b
:102760000400fa00889fbe008a9fbe008c9fbe00b6
:1027700080bf9f0091bf9f000206be00e7020700d6
:102780000001be000004be000c00be00dd05070015
:102790000fb997009fb99700000551008185590036
:1027a0000800be000a01be004f06be004f05be0075
:1027b0004f04be000080fa00000006000a00fa0084
:1027c000889fbe008a9fbe008c9fbe0000047800d8
:1027d00001457800820578008304780004067800bb
:1027e0000300e00002003c0019002000abca2000fa
:1027f00060c6b300804f55000e00320060c4b300c5
:10280000804f55000b00320070c6b300804f55005a
:102810000300320070c4b300804f550083003a00bb
:10282000e40f46008100350058089000800f5600e4
:102830007e003d000c06e80060c6b300804f5500e6
:102840001000320060c4b300804f55000d0032000c
:10285000081090000038a30004003a0058089000c7
:10286000808f540001003d00590c980058089000da
:102870000c005000500c980002003b000000eb00e0
:10288000500c98000c00e00027003c00f2014400ce
:10289000130178006800900001c3b3000170790053
:1028a0000201e80082097800580890000000e0006a
:1028b00003003c00081090000038a3000400320020
:1028c000e8009000e0c2b300807079008209e8005f
:1028d0000c00ea00d8089000808f500001003d00f5
:1028e0000106ea000c00ea00200c98000c80400071
:1028f000500c9800890f500001003d0080047800c2
:10290000680090009808900001004000390c980081
:10291000090178008b00780008f70700580890003c
:10292000090050001a003700e800900018089000d5
:102930008c8f540018003d00008040000901780091
:102940008b007800fdf60700180890000901400090
:10295000120c980009005600200c980058089000ae
:102960000000e00003003c00081090000038a300c5
:1029700006003200e8009000e0c2b30080707900e9
:10298000380890000000e800300c980058089000cb
:10299000400c9800a3003700008040000c01780034
:1029a0008b007800e5f60700180890000c00400046
:1029b000100c98008c845400580890000000e0002f
:1029c00003003c00081090000038a300060032000d
:1029d000f20144009300780068019000e0c2b30067
:1029e00000f178008109e80058089000890f500034
:1029f00001003d0080047800680090009808900075
:102a0000010040008c80450009017800cbf60700ea
:102a10001808900009004000100c98005808900019
:102a200009005000200c98007e00370070c6b300eb
:102a3000804f55000300320070c4b300804f550032
:102a400014003a0058089000808f540004003d00a4
:102a5000081090000038a30001003a00590c9800bb
:102a6000580890000000e900500c980002003b005c
:102a70000000eb00500c980051c6b30070c6b300c4
:102a8000804f55000100320051c4b3000145780069
:102a90000900370010c6b300804f550002003a000d
:102aa0000ac7b3000400370010c4b300804f5500bc
:102ab00001003a000ac5b300f20144001301780096
:102ac000680090003b7079000201e80082097800fc
:102ad000580890000000e00003003c00081090003f
:102ae0000038a30004003200e8009000e0c2b30008
:102af000807079008209e800580890000000e0002a
:102b0000100034008904e900890f500001003d00e5
:102b10008004780068009000980890000100400050
:102b2000090178008b00780084f6070018089000ef
:102b300009004000100c980058089000090050004f
:102b4000200c9800e8009000180890008085400054
:102b50008a5d78008b06e8000c00e0000400350078
:102b6000b0c2b300804d78008d05780004003700b6
:102b7000d0c2b300804d78008d0578000c06ea00c5
:102b80008004eb000c00e00009003400a1002000ec
:102b90000c0078008d0007007681540001f17f0061
:102ba000000678008904e8000000e000f7ff3c0020
:102bb000e18f540009003c0050c6b300804f55001f
:102bc0000300320050c4b300804f550003003a00a8
:102bd00000c3b300805e78008d0578000900e00036
:102be00002003a0000c3b300805d78000900e000f5
:102bf000070034008904e900f680540061c07f00ba
:102c000002c3b300825d40000900e000f9ff3c0010
:102c10006800900098089000010040000080550076
:102c2000300c98000810900074006000f00f500005
:102c30000e003a00780090009808900001004000d3
:102c4000a808900001004000b80890000100400072
:102c5000c80890008100400078089000808f5000e4
:102c600002003d0001005000000c98004f06be001d
:102c70004f05be004f04be000080fa0000000600b1
:102c8000000278003000900001002800010360007d
:102c9000150020006f0060003002980008003a0024
:102ca000240090000000e00005003a0014009000ad
:102cb0000000e00002003a001400e0003e00320094
:102cc000340090000000e0000b003a002400900067
:102cd0003002980014009000200298001400780040
:102ce00010029800000aeb00f082520034009000bd
:102cf0000000e000f5ff320034009000ef0f5000bc
:102d000014003e008001d000a40090004f08de00b7
:102d100080817100330298008100d000140190007e
:102d20004f10de0080807000210298000201d00068
:102d3000940078004f08de00000171001202980034
:102d4000010ad0008502e90003007800ef8f5100ee
:102d5000ecff3600b4019000ff8f510013003600e5
:102d60001401d10014009000cf00dd00010a7100b1
:102d70000000d100a40090004f09dd0002007000a7
:102d8000100298008100d1004f18dd008080700093
:102d9000210298000300d100300298008502e8006b
:102da00080017800ff0f5000edff3e0034009000de
:102db0006f00600030029800340090000600700040
:102dc000300298000500780000000600010178003c
:102dd00000027800110009000200d8000002fd0086
:102de0000491b900820250000400be0000000600f9
:102df0000a00fa0000027800c3202000e52020002d
:102e00000721200046212000e20f50001b003e0059
:102e100060638000e10f5000040032006321200055
:102e200085212000a7212000e621200013409000ea
:102e30000078a30002003a00000beb0013f0a000a2
:102e4000154090000028a30001003a0015a0a00042
:102e5000820178000200e00010003200154090006e
:102e60000008a300fdff32003100fb00800b78005a
:102e70008301e900f9ff3a00080037003000200024
:102e8000b0bf9f00c4bf9f00d1bf9f00e2bf9f00a3
:102e90006a80570000c0da006fb99700020078001e
:102ea0000080fa00000006000a00fa00110020006d
:102eb000b1bf9f00c0bf9f006a80570000c0da000a
:102ec0004fb897000080fa00000006000a00fa00e0
:102ed00051002000b1bf9f00c0bf9f006a80570013
:102ee00000c0da005fb897000080fa00000006001a
:102ef000889fbe00800478006e0ce20005003a0056
:102f00000000eb00100007008080eb000000e000f4
:102f10000a00350078638000880078000900e0002e
:102f20000600320009004400070007008080eb0023
:102f30000000e00001003500880078000100780002
:102f40004f04be0000000600800078000001eb0086
:102f50000000e00003003a00c0ca2000706388004f
:102f60000600370000ea2000808f500002003e007b
:102f700071638800010037000081eb0002007800d7
:102f800000000600889fbe008a9fbe0001057800f1
:102f90000100e0000400350008003c000000e000f3
:102fa000200032000500370060001000e0801800ab
:102fb00002003b0001f02c001a0037000004be00a4
:102fc0006011b8006b0920000982cf0002003900af
:102fd0000882cf000441b000694252000e00320066
:102fe00008003b0082817100610164008904d10006
:102ff0000884d3008b05e8000442e800f9ff3a009a
:10300000050037000804440089844c008b05e90062
:103010000442e900fbff3a00e20007000af0a700c3
:1030200001f0a0004f05be004f04be0000000600e6
:10303000889fbe008a9fbe008c1f7800ff0007009b
:103040000601330003866c006450e1002e0032005c
:103050006420e100330032006150e1002f003200b3
:103060006120e1003100320085855500eb07b0009a
:10307000090020000804200005003700080444006f
:1030800089844c000a0031000603430087834b000b
:103090000001530081815b00f8ff33000203be0092
:1030a0000800a0000804440089844c00f6ff3900a1
:1030b000c639dd00830173000100320013002000d7
:1030c0008904d1000884d3000998a30005003200c8
:1030d0000800a7000300a0008904d1000884d300e1
:1030e0008b05e8008904d1000884d3000001eb00bf
:1030f0000281d200ab00070001f0a1000cf0a70094
:1031000001f0a000de0037006420e100e0003200a2
:103110000801be000200be00f7ff37006120e10099
:10312000db0032006000b800f3ff37000000200031
:1031300001f82700f0ff370003f0a200889fbe00cf
:103140008a9fbe008c1f7800bc000700c3003300bc
:103150006450e1004f0032006420e1005200320070
:1031600003826c0007003b000905d0000306d00075
:10317000820f54000c065d0002003900020032008c
:1031800089017800030678008582550004003d001f
:103190000003fd008103fd008502ea008b854200eb
:1031a000840f720002003b0060001000e0801800f5
:1031b0006011b8000005eb007a28e1000a00390030
:1031c00006007800c75ddd00f707b2008780750054
:1031d0002d003700828171000a01780061056000ce
:1031e0008180d1000080d3008502e900f9ff3b0017
:1031f000060440008784480002003b00600414007d
:10320000e0841c000988a300070032008a81710055
:1032100082817100610164008904d1000884d300b7
:103220008b05e800170037000978a30013003a0067
:103230000b00e000130034008b05e9000804440093
:1032400089844c000a4474000978a3000d003a00f8
:103250000b00e000070034008b05e900080444007f
:1032600089844c0001003a000b0020000978a3007b
:10327000f7ff32000001eb0002003700828171008d
:103280000a017800470007000cf0a70001f0a00039
:103290007b0037006420e10002003a00838f6c005d
:1032a0007b0033000801be000200be00740037003e
:1032b0000001be00790007000470a70003f0a10020
:1032c00003f8a30013003a006509b10010003200b2
:1032d000090035006928e1000200350001002800de
:1032e0000000050000004000818048008502e900e0
:1032f000fcff3a0000000600f88f42000500350090
:103300008100d1000080d3008502e800fcff3a0074
:10331000000006008000eb0000000500839f6800ad
:103320000100e00002003d0060001000e080180095
:103330000300e00002003d0060011100e08119007f
:10334000050007004f00e00002003b006000100095
:10335000e0801800000006006022b800060220008d
:103360000000d0008180d2000482d2008582d20089
:103370000000a0000202520083825a0003003b00ba
:103380000202420083824a000000a1000603e90015
:10339000f3ff3a0000000600efff07000400be0044
:1033a0000000060081002000618055000b003d00f8
:1033b0000b00200061fe2f000100e1001d00340021
:1033c00082817100610164008904d1000884d30006
:1033d0000000e800faff3a0071002000610064007c
:1033e0000300700002006000090032006104440024
:1033f000e0844c000988a500050032008b05e80038
:103400006808e10002003a008904d1000884d30072
:10341000f20f20000258e10005003d00c75ddd000d
:10342000f907b200898075000800780000000600e6
:103430000bf827008b007800000005000004be0098
:10344000160007000003be000405be000200be0017
:1034500012000700844f7500000006000200be0045
:103460006450e100050036006420e10002003600ef
:103470000968a30001003a000800be000160a00036
:103480004f0678004f05be004f04be000000060046
:10349000f0ff2f00f1ff2700f9ff3700c70ade0019
:1034a000f107b200f50fb20008003200e1cf420090
:1034b000020032000170a00024000500810f70009e
:1034c000010032000408050044000500810f70006f
:1034d00002003a00140005008502e90000004000e7
:1034e00081c04800fcff3b000170a00024000500e3
:1034f00081037800e9ff07000001be006000b8000a
:103500000478a30013003a006220e10015003e0099
:103510000d0039008301d1000281d3008180d300e6
:103520008301d1000281d3008180d3008301d100c7
:103530000281d3008180d3000538b000c42add00a9
:10354000f300b2008381720007f0a70003f0a0002f
:1035500000000600f3ff2700f2ff2f006110b90002
:10356000fbff370003ff2700f7ff37006000100064
:10357000e080180060011900e081190000000600d9
:10358000881f7800000478005001be004000be0093
:103590000000420081804a0002014b0083814b0001
:1035a000009cbe000294be00dc0007000300310056
:1035b000480090000000e800400498004f047800a4
:1035c00000000600889fbe00000478008004eb0025
:1035d0005001be004000be00d000070001003100d5
:1035e0001900200004005000858058000601590091
:1035f00087815900009cbe000294be0048009000e4
:1036000009005000400498004f04be00000006006e
:103610001200fa00889fbe008a9fbe008c1f7800af
:103620000205be000004be00f4b79f0085bf9f00e6
:1036300096bf9f00a7bf9f000000eb00e0b79f0070
:10364000d0b79f00c0b79f00b0b79f00a0b79f0042
:103650000006eb005fb197006fb097008000d000cc
:103660000000e00015003d00e1b79f000100780078
:103670000200e00001003d000000a000ac000700d7
:1036800001003d000000a000af00070001003d0068
:103690000000a000b200070001003d000000a000f3
:1036a0008100070001003d000000a000b2000700fb
:1036b0007c805700b2ff070014003700e1b79f007d
:1036c000010078000200e00001003d000000a000c1
:1036d0009700070001003d000000a0009a000700cd
:1036e00001003d000000a0009d00070001003d001a
:1036f0000000a0006c00070001003d000000a000d9
:103700009d0007007c805700aeff07006fb0970058
:103710000000e0000700350010002000010020003c
:103720006011b80008047000898470000a057100f7
:103730008b8571000c06e800f0032000800f560016
:10374000c4ff34006fb097000000e00006003d00a9
:103750007fb297008fba97001fbb9700afbb97004f
:103760007c80570086ff07000802be000a03be00e7
:103770006fa897000000e00004003a002fb2970005
:10378000bfb297004fb39700dfb397000400be00ad
:103790000601be004f0678004f05be004f04be0074
:1037a0000080fa0000000600881f78001800200042
:1037b000881f780096ff07008f87e9004f04780084
:1037c00000000600801feb0091ff07008f87e900d3
:1037d000000006000800fa00889fbe008a9fbe0015
:1037e0008c1f78006e00070005003d0043000700b5
:1037f000300007000c003d00330007000b003700cd
:10380000e00f5200e08f5a00e00f5b00e08f5b009a
:1038100006003d000400be000601be0053ff070085
:103820000205be000004be001c0020002c000700a2
:10383000ddff07000c00e000010032004bff070035
:103840004f0678004f05be004f04be000080fa000e
:10385000000006000800fa00889fbe008a9fbe0094
:103860008c1f78004e00070002003d001c00200065
:10387000220007000f00070001003d0012000700b2
:1038800017000700cfff07000c00e0000100320026
:1038900036ff07004f0678004f05be004f04be00fc
:1038a0000080fa000000060090b79f000100d000e1
:1038b00080b79f00e00f5400e08f5c00e00f5d00d8
:1038c000e08f5d00000006000800be000a01be0097
:1038d00026ff07000205be000004be00000006002f
:1038e0000802be000a03be005fb09700efb0970069
:1038f0007fb197008fb99700000006001bff0700fb
:103900000100070000000600b0b79f00c1b79f008c
:10391000d2b79f00e3b79f00000006000400e1005b
:103920000588e1000690e1000798e100000006002c
:10393000c0b79f000200d000b0b79f00afb09700a3
:103940000100e00000000600b0b79f000100d000b9
:10395000a0b79f009fb097000100e00000000600a4
:10396000a0b79f000100d00090b79f008fb09700d4
:103970000100e0000000060080b79f000804d000ae
:103980008984d2000a85d2008b85d2005fb297006d
:10399000efb297007fb397008fbb9700000006003f
:1039a000d9ff07000605be000404be000006eb00b8
:1039b000e00f5000e08f5800e00f5900e08f5900f1
:1039c00000000600889fbe008a9fbe008c9fbe003c
:1039d0000404b8000506b8008904460060854e005e
:1039e0000606b8000a054600e0854e000706b80046
:1039f0008b054600040eb800890446000a854e0077
:103a0000050eb8000a0546008b854e00060eb8006c
:103a10008b0546000416b8000a0546008b854e004b
:103a20000516b8008b054600041eb8008b0546003d
:103a30000800be000a01be004f06be004f05be00d2
:103a40004f04be00000006000800fa00889fbe0078
:103a50008a9fbe00170007000605be000404be00d2
:103a6000e00f5200e08f5a00e00f5b00e08f5b0038
:103a700008003d000400be000601be00bbfe0700ba
:103a80000205be000004be000f000700b7fe0700dd
:103a9000080007000802be000a03be000a00070073
:103aa000c8ff07004f05be004f04be000080fa00ab
:103ab00000000600e0b79f00f1b79f0082bf9f00a3
:103ac00093bf9f00000006006fb09700ffb0970003
:103ad0000fb997009fb99700000006008f1fd10013
:103ae0000e0107008f87e9000000e00000000600db
:103af0001400fa00889fbe008a9fbe008c9fbe0003
:103b00000004be000205be00680047000a90be0027
:103b10000890be002a0107000070a7000bf0a1006a
:103b2000304320009e02900080825200b0fe2f00a1
:103b30000028e10011003d00b0fc2f000028e1004a
:103b4000150034001e0990008e0890007e00900041
:103b50000501b0000201d1008180d3000080d300b4
:103b60008502e800fbff3a000b00e0004f013b003c
:103b700060001000e08018004c013700f0ff2f00bb
:103b8000f1ff27000b00e00048013b000100280086
:103b900000002000450137006000b80043013700f5
:103ba0004f89de00820178004501370007f0a2004e
:103bb0007a013700809feb00d80007008f87e9006b
:103bc0000000e000000006002800fa00889fbe0008
:103bd0008a9fbe008c9fbe0003866b001f010700fa
:103be0000028a30064003a000128a30067003a00ff
:103bf0000008a30062003a000108a30065003a0033
:103c00001e009000be08900081064000ed3fb1000c
:103c1000f4805700ee019000111ab8008e09900050
:103c2000311bb8009e099000311cb800511db8002e
:103c3000f485570046000700fe0190003a00070097
:103c40008b85e8003e0007008e09900040000700c9
:103c5000ee019000340007008b85e8003800070073
:103c60008e099000400007009e0990001b18b800c4
:103c7000890440000a854800fe01900034000700d6
:103c80008b85e80038000700ee0190003000070047
:103c90008e0990001b18b800890440000a8548006e
:103ca0000a98a30008003a000402420085824a00f4
:103cb00006034b0087834b0008044c0089844c00aa
:103cc0000a054d008d06e9008482720085027300aa
:103cd0004c3add0085027200010032001500200020
:103ce000443ade001400b2004538de00cb45dd006a
:103cf0000b007000c540de00cb4ddd008b807000f6
:103d00004549de00cb55dd000b017100c551de00d9
:103d10000d0378009e01070003f0a1000cf0a7003e
:103d200003f0a000e10037001b18b8008502400036
:103d300006834800e0834b0060044c000700370016
:103d40001b18b8000603400087834800faff3700bd
:103d50001b18b8008703400008844800e0844c002a
:103d600060054d00000006001b18b8000804400064
:103d700089844800faff37000108a300c8003a0010
:103d80005800be005801be00e3ff37000008a30042
:103d9000c3003a0009047800f9ff37002800fa0050
:103da000889fbe008a9fbe008c9fbe0003866b006a
:103db000aa0007006400e100440032006408e1004a
:103dc0004a0032006100e100460032006108e10073
:103dd00049003200ec0647006000b8003d02be001a
:103de0003d03be00f48657006011b8003d04be00dc
:103df0003d05be007d0320000b0037000000a00041
:103e00008d06e900130032000402420085824a0058
:103e100006034b0087834b00000040008180480070
:103e200002014900838149000802520089825a0038
:103e30000a035b008b835b00f0ff3b00080242003b
:103e400089824a000a034b008b834b008d06e900f0
:103e5000edff3a008482720086827200f707b2009a
:103e60008782720001003200150020001e049000bd
:103e70003e0b900006035400e63fb0000368a30029
:103e8000070032000000a7000500a0008301d10058
:103e90000281d3008180d3000080d3000603e800b4
:103ea0008301d1000281d3008180d3000080d30040
:103eb0000002eb000482d2003501070003f0a100ec
:103ec0000cf0a70003f0a000780037006402470060
:103ed0006408e100720032003400be003401be000c
:103ee000f6ff37006108e1006d0032006011b80094
:103ef0006000b800f1ff370003ff27000200200038
:103f0000fbff3700020ab900001bb9000200b8002d
:103f1000810042008100430000000600889fbe002f
:103f20008a9fbe008c9fbe000404be000605be0032
:103f3000809fbe00829fbe004101070004067800fa
:103f40000800be000a01be003d010700840678009b
:103f50004f03be004f02be008d4f76007fb097002a
:103f600013003300f0ff2f008b8f6b0006003b0027
:103f70000d0666000c00a7000a00370007f0a60037
:103f8000100020000a003700880f5200898f5a0065
:103f90008a0f5b008b8f5b0003003900100020004c
:103fa00001003e000000200007f0a7000000ea002a
:103fb0004f06be004f05be004f04be0000000600c5
:103fc000800078005002be005003be004439de007d
:103fd000f700b200f37f2000030161000900320006
:103fe0000218e10016003a00850172008301730097
:103ff000838173000008200015003a004000200073
:104000001300370085017200830173008381730000
:1040100005003a0004a8be0006a8be00100020005b
:104020000b0037000201e9000402420085824a00c9
:1040300006034b0087834b000748a300f9ff3200bb
:104040000740a00004a8be0006a8be002000200073
:104050008000980092009800000006006804470065
:104060000294be000094be00fc0447008694be008b
:104070008494be0009007800d1ff07000800780092
:10408000cfff070099007800814f70000b003b00c4
:104090000800be00fc0007004f00b100030037001d
:1040a000f3ff2700f2ff2f006110b9004f06be009a
:1040b0004f05be004f04be000080fa00000006005d
:1040c000889fbe00830478000300e0002c003500c8
:1040d00003003c00008270000402710026003200e0
:1040e00036432000c50020008383cf000a0039003a
:1040f0000541b1008283cf00070039000541b100be
:104100008183cf00040039000541b1008083cf00d6
:10411000010039000541b10085c353006022b80099
:10412000120032000a003b008482720061026000cb
:104130008301d1000281d3008180d3000080d300ad
:104140000603e8008743e800f7ff3a00070037005e
:10415000000040008180480002014900838149003d
:104160000603e9008743e900f9ff3a0088000700e9
:1041700009f0a70003f0a0004f04be0000000600f5
:1041800060001000e080180060011900e081190053
:10419000d3ff3b00033e2c00f7ff37002800fa0056
:1041a000889fbe008a9fbe008c9fbe0007067800d5
:1041b000878669000c003b000304780087047800c0
:1041c00008f0a10009f0a100840f5000858f58006d
:1041d000860f5900890f5c00030033000cf0a20029
:1041e00001003a000cf0a1009cff07006400e10010
:1041f0005f003200780147006408e100610032008e
:104200006c014700748557003200be001201be00e9
:104210003a04be001a05be001e039000be0a9000bc
:104220008503530006003d000004fd008104fd00ed
:104230000205fd008305fd008703ea000503780001
:104240000df8a3000400320060041400e0841c0098
:1042500060051d00e0851d006022b8007d03200080
:104260000d38e1008006eb000b0039004433dd001f
:10427000f300b200830173003900370084827200ba
:104280000d027800e10664008b85d1000a85d30019
:104290008984d3000884d3008703e900f7ff3b003b
:1042a00008004000898048000a0149008b814900cc
:1042b00004003b0060001000e0801800600119005d
:1042c000e08119000358a300090032008d827200ba
:1042d00084827200610260008301d1000281d300f8
:1042e0008180d3000080d3000603e8001b00370064
:1042f0000348a30017003a000600e000170034004e
:104300000603e9000d00a30000004800818048007a
:1043100002014900838149000348a3000f003a00cd
:104320000600e000090034000603e9000000400038
:1043300081804800020149008381490001003a0060
:104340000003eb000348a300f5ff32006022b80031
:104350000200370084827200618266000c00070050
:1043600003f0a1000cf0a70003f0a0004fff3700fe
:10437000640147006408e10002003a000df8a30060
:1043800047ff3a003200be001201be0047ff37006f
:104390001800200057002000080453000d003d00c5
:1043a0000600200097fc2f000740e1001e003400ab
:1043b00084827200610260008301d1000281d30017
:1043c0008180d3000080d3000804e800f8ff3a00a1
:1043d00047002000610460000504740004046400c8
:1043e0000d00320061004000e0804800600149009b
:1043f000e081490003b8a500070032000603e80089
:104400006538e10004003a008301d1000281d30045
:104410008180d3000080d300f87f20000830e100c5
:1044200003003500080378006000b8006011b80090
:104430004433dd00f300b200830173000000060086
:1044400005ff270005826100070032000428e10013
:1044500001003200240005000600070001003a00b8
:10446000440005000408050002000700f9ff3a00b7
:10447000140005006f8261008102700085027100e6
:104480008502720000000600e48240001078a3005c
:1044900007003200640240001178a3003400be001f
:1044a0001401be00040032000330a7000000060023
:1044b0003500be001501be000330a000000006005c
:1044c0000000fa000000eb0050158800f01f2800e3
:1044d00040158800e000200030158800000820000a
:1044e000201588000000eb0010158800000028004f
:1044f000001588000080fa00000006000200fa00a3
:10450000000f78009e0078006f80600030158800f2
:10451000a022a800401f200009110700a022a90026
:10452000a0c2bf000080fb00610060000000e0004e
:10453000fbff3200001480000080fa00000006003b
:104540000000fa0051428000400020000008b8003e
:10455000c2972000020040001000be0089fa070048
:104560000200200003d82400b1fa0700104d880093
:10457000214d88000080fa00000006000800fa00c3
:1045800051428000400020000008b800a2942000a2
:10459000020040001001be00200020000012b80000
:1045a000048fbe000000eb000092b9009e00900056
:1045b00084804000030078000000d000808040002c
:1045c000110798001e00be00e00f5000e08f580059
:1045d000050035001e00be006afa0700200798009b
:1045e00031079800120037001e01be006100610013
:1045f0008000eb001e02be008501d1000481d300c3
:1046000002007000838070005efa070020079800a7
:10461000310798002e019000be0190002e009000fe
:10462000be009000c5fa07002007980031079800e7
:10463000124d8000234d80002e009000be0090009f
:104640007bfa07001afb0700f04c8800014d880038
:104650000080fa00000006000000fa00c7ff070013
:10466000f04c8000014d8000341307000080fa00f8
:10467000000006000400fa000000eb00d04b8800a8
:104680000000eb00000f7800800120009e0f10005a
:1046900024003e00710120009e8f100008003e00a3
:1046a0001e0078000000d000a2942000820040008c
:1046b000d04b800011004000d04b88000300370031
:1046c000d04b80000000ea00d04b88001e0078002c
:1046d0000000d00002002f008200400012002000e5
:1046e000f0072000b5120700100798001e007800a0
:1046f0000000d00001002f00010140001e007800e2
:104700000000d000a1942000010040001300200010
:10471000f1072000ca120700100798001e0fe800da
:10472000d9ff3700304b8000e10f500009003a00fc
:104730007a09f8001e019000821f78001e007800a0
:10474000801f780020df2d00801f78001bef0700fe
:10475000e88757000080fa00000006000600fa0013
:104760000000eb00200798000000eb00000f78002d
:10477000800120009e0f100015003e001e007800f2
:104780000000d000a1942000010140001e0078002c
:104790000000d00003002f00830040001300200021
:1047a000f007200078120700100798001e0078001c
:1047b0000000d000a2942000820040002e00900053
:1047c00011004000200798001e0fe800e8ff3700a6
:1047d0001300200082942000010f2f00f00720001a
:1047e000691207002e0090000080fa000000060009
:1047f0000400fa000000eb00e04c88000000eb0031
:10480000000f7800000120009e0f100024003e00e1
:10481000f10020009e8f100008003e001e0078006e
:104820000000d000c297200082004000e04c8000d1
:1048300011004000e04c880003003700e04c80008d
:104840000000ea00e04c88001e0078000000d00064
:1048500002042f008200400012002000f007200018
:1048600056120700100798001e0078000000d000c4
:1048700001042f00010140001e0078000000d0005c
:10488000c19720000100400013002000f107200024
:104890006b120700100798001e0fe800d9ff3700c1
:1048a000304b8000e10f500009003a009c09f800ed
:1048b0001e019000821f78001e007800801f780083
:1048c000b0e12d00801f7800bcee0700e88757009c
:1048d0000080fa00000006000600fa000000eb006d
:1048e000200798000000eb00000f78000001200076
:1048f0009e0f100015003e001e0078000000d00042
:10490000c1972000010140001e0078000000d00087
:1049100003042f008300400013002000f007200054
:1049200019120700100798001e0078000000d00040
:10493000c2972000820040002e009000110040002d
:10494000200798001e0fe800e8ff37002e009000b7
:104950000080fa00000006000600fa000000eb00ec
:10496000000f7800f00e20009e0f10000f003e0098
:10497000640147001e0078000000d00003102f00e3
:104980008300400013002000f0072000fe11070004
:1049900010079800818520001e804000ce419000c5
:1049a000034878001e0fe800eeff37000080fa0091
:1049b000000006000600fa000000eb00000f78007f
:1049c000f00e20009e0f100017003e008185200091
:1049d0001e8040001000fb00200798001e00780099
:1049e0000000d00002102f008200400012002000c2
:1049f000f0072000f1110700100798001e00780052
:104a00000000d00001102f000101400064004700a9
:104a100013002000f107200009120700100798007a
:104a20001e0fe800e6ff37000080fa0000000600d5
:104a30000200fa00003e290041002000504a880090
:104a4000614a880000122a0071002000704a880024
:104a5000814a88000034210021002000904a88000b
:104a6000a14a88000000eb00b04a8800800c2000ba
:104a7000e04a88000000eb00c04a88000000eb001c
:104a8000d04a88000000eb00a04b88000000eb003b
:104a9000b04b88000000eb00904b88000000eb005a
:104aa000c04b880020002000004b8800c02b200055
:104ab000f04a8800007d2000104b8800400620004e
:104ac000204b880010002000304b88003000200070
:104ad000404b880080bb2000504b8800c05d200008
:104ae000604b880080252000704b8800c012200099
:104af000804b880070682d0021012000e04b880069
:104b0000f14b880000d82800b1052000004c880037
:104b1000114c880000d0220011132000204c880086
:104b2000314c880000fa200001002000404c880031
:104b3000514c88007008200001002000604c880063
:104b4000714c88004001200001002000804c88004a
:104b5000914c88004001200001002000a04c8800fa
:104b6000b14c880020032000c04c88007000200059
:104b7000d04c88000000eb00000f7800f00e200001
:104b80009e0f100006003c00808520009e00400023
:104b90000040eb00804878001e0fe800f7ff370068
:104ba00050e42d00801f780080852000e4ed070090
:104bb0008f87e9007fff0700130020008294200008
:104bc000010f2f00f00720006f110700404a8000fe
:104bd0000000e800404a880012002000010f2f006a
:104be000f00720007511070013002000020f2f00ae
:104bf000f107200080942000911107000080fa0046
:104c0000000006000e00fa00000f7800110798005f
:104c10009e00900040062000008ab9001e00780027
:104c20006101b9000400be00bcf90700300798001c
:104c30004107980042062000030020003e0090003b
:104c4000ce0090000000510081805900500798006c
:104c5000610798005e009000ee009000e00f5000a9
:104c6000e08f580004003c001000200001002000ec
:104c70005007980061079800100320009e0f100055
:104c8000150034003e009000ce0090004206200047
:104c90000202b8000001eb000283b90005017800b0
:104ca00006014100430620000388b90000014100cd
:104cb0008202780000712200010020000400400000
:104cc000858048005e019000ee01900093f9070096
:104cd00020079800020037000000eb002007980032
:104ce000ae009000f0702200808f5000020034006f
:104cf000f0702200200798002e0090000080fa003b
:104d0000000006000200fa00b04a8000000f7800a0
:104d10001e007800e10f5000110032001e007800e4
:104d2000e10f500004003c001e0078000000e0008d
:104d300008003200130037001e007800e20f500018
:104d40000a0032001e007800e30f50000a00320013
:104d50000c00370000e62d00941307000b0037000d
:104d600080e62d00911307000800370000e72d00b2
:104d70008e1307000500370080e72d008b13070016
:104d80000200370000e82d00881307000080fa00b9
:104d9000000006000000fa00a40be20005003a0043
:104da00080e82d00811307000000eb00804288009e
:104db000170037005008e20005003a0010002000fc
:104dc00080428800e1012000f0a42000b50c07001b
:104dd00070428000620060000000e00003003200ca
:104de000e0e82d00711307000900370070428000d1
:104df000640060000000e0000300320040e92d0084
:104e00006a13070002003700a0e92d0067130700ae
:104e10000080fa00000006000200fa004141800014
:104e2000201c21000088b9004108de00010020009c
:104e300040428800404280004f1207000080fa0084
:104e4000000006000600fa004c08e2003f003200b5
:104e5000e2418000f3418000004280001142800066
:104e6000800f5100818f590007003400e04180001d
:104e7000f14180000042880011428800e0152000c6
:104e8000405d88001b003700a80be20019003a00c3
:104e900020032000405d8800004280001142800015
:104ea0008180d1000080d30010079800210798006e
:104eb0001e009000ae009000e00f5000e08f580000
:104ec00004003a006000b8000042880011428800e7
:104ed0000800370000428000114280001e0190004f
:104ee000ae0190000200500083805800004288000c
:104ef0001142880000ea2d002c13070001428000b7
:104f0000a04c8000000ab80001428000b04c800034
:104f10000088b9000501780000014100a14c800023
:104f2000104280000088b900000141008202780030
:104f300040a8de00cf80de00000f7800710720005f
:104f40001e007800d1140700040037006dff070031
:104f50006000b80000428800114288000080fa001a
:104f6000000006000000fa004c08e20018003200c1
:104f70009000200061fd0700cf80de00424c8000e1
:104f80000202b800524c80000283b900050178008b
:104f900006014100434c80000198b9000001410026
:104fa0008202780040a8de00cf80de0060418800e9
:104fb00040ea2d00fd120700110020006041800032
:104fc000b214070060ea2d00f81207000200370053
:104fd00080ea2d00f51207000080fa0000000600ac
:104fe0000000fa00c14c8000c0f620002d0c070024
:104ff00035110700004b2000305d8800d4c2bf008f
:105000000080fb0061006000e10f50001e003a00cc
:105010000040eb0022110700305d8000c21220002a
:10502000110009000280d800801f780000eb2d00dd
:10503000801f780040802000c1ec0700e487570003
:1050400040802000d912070000c4b30014110700eb
:1050500030ec2d00d5120700a60be200e7ff3a0066
:10506000c04c80008000d000e02521000d0c07001e
:10507000d4c2bf000080fb0061006000e10f50005f
:10508000fbff3200ddff3700a60be2000c003a0008
:1050900078fd0700304b8000e10f500004003a001b
:1050a00040ed2d00801f7800c4ec07008f87e900d9
:1050b00020002000500e0700cfa2a900ffff3700fc
:1050c0000080fa00000006000000fa00e7c2bf00fe
:1050d0000080fb004700de000080fb000000e000d5
:1050e00004003200c4c2a900704280000020a00069
:1050f00070428800b04a80000000d000a2962000d4
:105100008200400020428000910f50000b003400cc
:10511000b04a80000000d000a2962000820040002b
:1051200030428000910f500004003400c4c2a90036
:10513000704280000010a000704288004e08e2001b
:10514000060032000000eb00c04088000000eb00c9
:10515000904b88000000eb00b04b88000080fa0004
:10516000000006000000fa000000eb00704288001a
:105170000000eb0080428800caa2a9004001200084
:105180001d0e0700caa2a8000080fa000000060059
:105190000000fa00e04a8000e90f500007003c00e0
:1051a0005c09f80010f02d00801f7800408020007e
:1051b00063ec0700e48757000a003700e04a8000ec
:1051c000a2002000110009000200d800801f780012
:1051d00090f02d00801f78004080200058ec0700e0
:1051e000e487570040802000701207000080fa001a
:1051f000000006000200fa00b310070000f12d00c5
:105200006a12070000c4b300a510070010f22d00b9
:1052100066120700130f07000004e00011003200bf
:10522000200f0700004f7800a1002000f0a420000c
:105230009c0b07001e407800fb0e070000c4b30063
:105240009710070020f32d00581207001e80fb0066
:105250002f120700c0f32d00541207001e407800e3
:1052600031120700d4c2bf000080fb006100600063
:10527000e10f5000e7ff3a000080fa00000006004e
:105280000400fa00b00020009cfc0700000f78002a
:105290000000eb0010079800f02820009e0f10007f
:1052a00005003400603d20009e0f100002003c000d
:1052b0001000200010079800205c20009e0f1000b6
:1052c00005003400907020009e0f100002003c008a
:1052d00020002000100798001e0090000080fa00b7
:1052e000000006000200fa00b04a8000000f7800bb
:1052f0001e007800e10f50000c0032001e00780004
:10530000e10f5000060034001e007800e20f50004c
:10531000090032001e007800e30f5000090032003f
:10532000e802a900e822a90008003700e802a80066
:10533000e822a90005003700e802a900e822a80039
:1053400002003700e802a800e822a8000080fa0066
:10535000000006000000fa005809e20002003a00ce
:10536000e9a2a900cbc2a900c04a8000e10f500009
:1053700002003a00e9a2a800cbc2a900c04a8000fe
:10538000e20f500002003a00e9a2a800cbc2a80038
:105390000080fa00000006000000fa00d04a8000f9
:1053a000e10f500002003a00e9c2a80001003700f6
:1053b000e9c2a9000080fa00000006000000fa001f
:1053c00000ee2200e24a8000110009000200d8002d
:1053d000005d88000080fa00000006000000fa006e
:1053e000f04a80000000d0006101b90000002800f0
:1053f00001072000d8f70700904288000080fa00db
:10540000000006000000fa00d00020003bfc07006e
:1054100040418800c000200038fc0700504188004f
:1054200041418000404180000088b900a0418800cf
:10543000b141880051418000504180000088b9008e
:10544000c0418800d1418800a2418000b341800062
:10545000c0418000d141800000005100818059008e
:10546000e0418800f14188002042800030428800fd
:105470005141800040418000e2fd07002042880049
:105480000080fa00000006003400fa00889fbe0089
:10549000f0f32f00001688000000eb0010168800c3
:1054a00080e02300301688000000eb0040168800e2
:1054b000e0012400601688000000eb0070168800f0
:1054c00010002000901688000000eb00a016880055
:1054d000c0d72f00f01688000000eb0000178800ee
:1054e00000002800201788000000eb00301788001b
:1054f000cfa2a80040062000005d88008085200023
:105500000d15070040442500a00488009b0a0700f1
:10551000c0cc210000408800f30f07003c100700ba
:10552000240e0700e6fb070055ff070050428800e5
:10553000e50f070050428000600f9800ee089000d1
:10554000e18f5000070032006e099000e10f51001a
:105550000a003400ee099000e28f5100040032008e
:105560000600370010f42d009011070005003700e9
:10557000d0f42d008d1107000200370090f52d00aa
:105580008a11070080d82d008811070000c4b300dd
:10559000c30f070050f62d00841107000000eb0038
:1055a000f040880080bb2000305d8800d4c2bf007e
:1055b0000080fb0061006000e10f500019003a001c
:1055c000a60be200f9ff3a00c1122000e0252100fd
:1055d000b40a070000c4b300b10f070060f72d0044
:1055e0007211070010002000f0408800d4c2bf00f4
:1055f0000080fb0061006000e10f5000fbff320003
:105600000040eb00a60f070070f82d00671107009f
:1056100000c4b300a20f070080f92d00631107003a
:10562000e2ff3700acfc0700300798004bfc070096
:1056300040079800304b8000e10f500009003a000d
:105640004809f8004e029000841f7800be029000c6
:10565000851f780090fa2d00801f780057eb070017
:10566000e88757003e0090000000e00003003a0089
:105670004e0090000000e000080032006f050700b7
:1056800000ff2d00801f78004ceb07008f87e9009a
:10569000e7fc070056fc0700f6fb0700104b8000f4
:1056a000640a0700204b80005c0a07000000eb0042
:1056b000c04088000000eb00d0408800c04c800053
:1056c0008000d000f0a42000760a0700caa2a9003a
:1056d00010002000c80c0700caa2a8001e08e200a3
:1056e00001003200ec07070000000000cec2bf003e
:1056f0000080fb004400de000080fb0061006000d1
:105700000000e00012003a000040eb00640f0700c8
:1057100010022e002511070000c4b300600f07001f
:1057200020032e0021110700c3c2bf000080fb0030
:105730004400de000080fb00610060000000e0002b
:10574000eaff3a00bafc070029fc0700c9fb070082
:1057500040012000a80c0700404b8000a30d07006b
:10576000304b8000e10f500042003a005042800070
:10577000700f9800fe089000e18f50000700320083
:105780007e099000e10f51000e003400fe099000e8
:10579000e28f5100060032000a00370030042e006c
:1057a000801f780005eb07008f87e90009003700ac
:1057b00050052e00801f780000eb07008f87e9005e
:1057c0000400370070062e00801f7800fbea0700f7
:1057d0008f87e90080d82d00801f7800f7ea070046
:1057e0008f87e900a0082e00801f7800f3ea0700e9
:1057f0008f87e900e0d82d00801f7800efea0700ce
:105800008f87e900e0082e00801f7800ebea070090
:105810008f87e9000008f800600b2e00801f7800d9
:10582000e6ea0700e4875700404b8000e30f500092
:105830000b003200414b8000800020000008b800bf
:1058400094d92d0000004200801f78006809f800fc
:10585000e00c2e00801f7800d8ea0700e68757008a
:105860009a09f800800f2e00801f7800d3ea070005
:10587000e4875700c3c2bf000080fb004500de0084
:105880000080fb00610060000000e00001003a00c1
:1058900058fe07000000eb00e04088000000eb002d
:1058a000c0408800e842a900e862a900e9c2a90056
:1058b000c4e2a90022fb070030fb0700ba0e070074
:1058c0006000b8009d0e0700d04c8000cf80de0045
:1058d000c05c8800d15c8800b8fe0700bffe0700ee
:1058e0001dfc0700007d2000430c07004a08e20071
:1058f0000f003a0080112e00801f7800afea0700e9
:105900008f87e90000c4b300e50e070050152e0094
:10591000a6100700cec2bf000080fb004400de00de
:105920000080fb0061006000e10f5000f9ff3200d1
:10593000e50e07008002eb0005179800cac2bf0001
:105940000080fb000000d1000080fb0061006000cf
:105950000000e00002003a0010002000001798004c
:105960008e60900061c060000041d000a12c20003a
:1059700091407800d0cfb30000c0600002407000ba
:10598000cae2b700e8c2bf000080fb004200de00b0
:105990000080fb00610060000000e00003003200b6
:1059a0001000200060428800020037000000eb0079
:1059b00060428800c4fd07007209e2000300320063
:1059c00010002000a0428800020037000000eb0019
:1059d000a0428800904b8000e20f500003003a0084
:1059e00030002000b042880002003700024b8000e7
:1059f000b242880083fe0700c3c2bf000080fb00e4
:105a00004500de000080fb00610060000000e00057
:105a100051003a00803e2000305d88001808e20006
:105a200007003a00d0408000e30f500004003a0025
:105a3000c14c8000e04921009a0907000d003700a1
:105a4000c0408000e10f500007003a00e0408000b5
:105a5000ea0f500004003a00c14c8000e0492100e8
:105a60009009070003003700c14c800020f7200098
:105a70008c09070000000000c3c2bf000080fb00cb
:105a80004500de000080fb00610060000000e000d7
:105a900008003a00a60be200f7ff3a00c14c800074
:105aa000a00020000088b90080007800e0492100b3
:105ab0007c090700a60be20011003a00c0408000fc
:105ac0000000e800c0408800c0408000e10f5000a6
:105ad000020034000000eb00c0408800000000001d
:105ae000c3c2bf000080fb004500de000080fb0059
:105af000610060000000e000f9ff32001300370091
:105b00001808e20009003a00d04080000000e800d8
:105b1000d0408800d0408000e30f50000b003400dc
:105b20000000eb00d040880008003700e040800013
:105b30000000e800e0408800e0408000ea0f5000ec
:105b4000020034000000eb00e0408800c3080700ba
:105b500040062000a80b0700cec2bf000080fb005b
:105b60004400de000080fb00610060000000e000f7
:105b700062003a00803e2000305d88004e08e2005e
:105b8000060032000000eb00904b8800c14c800002
:105b900040882100430907004e003700934b8000e6
:105ba000131798001e129000e10f520012003200ed
:105bb0009e129000e18f520004003c001e109000e5
:105bc0000000e000080032000e0037009e10900038
:105bd000e28f50000b003a00c14c80004088210049
:105be0003009070007003700c14c8000e049210060
:105bf0002c09070003003700c14c800020f720006b
:105c00002809070000000000cec2bf000080fb0092
:105c10004400de000080fb00610060000000e00046
:105c200008003a00a60be200f7ff3a00c14c8000e2
:105c3000a00020000088b90080007800e049210021
:105c400018090700a60be20011003a007609e200ed
:105c50000c003a00904b8000e10f50001d003a000c
:105c6000004b8000e40f50001a003a0080852000ad
:105c7000311307000080eb00b04b88007dfa07006d
:105c8000140037000000eb00b04b88001100370013
:105c9000904b80000000e800904b8800904b800003
:105ca000e30f500002003a000000eb00904b880028
:105cb000904b8000e10f5000060032007609e200b0
:105cc000040032000000eb00b04b88000000eb0045
:105cd000904b880040062000470b0700cec2bf0053
:105ce0000080fb004400de000080fb0061006000db
:105cf0000000e000f9ff32001afd0700cec2bf002d
:105d00000080fb000000d1000080fb00610060000b
:105d10000000e00048003a00c3c2bf000080fb0062
:105d20004400de000080fb00610060000000e00035
:105d30000f003a0051428000400020000008b800e7
:105d4000a394200003014000514280004000200045
:105d50000008b800a494200004004000440620007d
:105d6000050020003019420020914a000e00370043
:105d700051428000400020000008b800a594200097
:105d80000501400051428000400020000008b8009a
:105d9000a394200003004000a40020000500200080
:105da0003019420020914a005142800040002000fa
:105db0000008b800a59420008501400062de2d0097
:105dc00051428000400020000008b800000041005f
:105dd0001302be00b00f5200a08f5a001000360010
:105de00051428000400020000008b800a594200027
:105df0008501400062de2d005142800040002000fd
:105e00000008b800000041001002be008489be00f6
:105e1000c14c800060042200a20807000300370084
:105e2000c14c800020f720009e080700d3f907002e
:105e300040062000f00a0700cec2bf000080fb0031
:105e40004300de000080fb00610060000000e00015
:105e500048003a00c3c2bf000080fb004400de00df
:105e60000080fb00610060000000e0000f003a00cd
:105e700051428000400020000008b800a594200096
:105e80008501400051428000400020000008b80019
:105e9000a494200004014000c0f92f00f1ff2f005e
:105ea000b2194000a29148000e0037005142800014
:105eb000400020000008b800a59420000501400023
:105ec00051428000400020000008b800a394200048
:105ed0000300400064ff2f00f5ff2f00301942003f
:105ee00020914a0051428000400020000008b80084
:105ef000a594200085014000a2dd2d0051428000c4
:105f0000400020000008b800000041001302be005d
:105f1000b00f5200a08f5a00100031005142800093
:105f2000400020000008b800a59420008501400032
:105f3000a2dd2d0051428000400020000008b80082
:105f4000000041001002be008489be00c14c8000e8
:105f5000600422005308070003003700c14c800092
:105f6000e04921004f08070084f90700400620009f
:105f7000a10a0700c3c2bf000080fb004400de008e
:105f80000080fb00610060000000e00041003a007a
:105f9000cec2bf000080fb000000d1000080fb00eb
:105fa00061006000e10f50003a003a00cec2bf002d
:105fb0000080fb004300de000080fb006100600009
:105fc000e10f500033003a00b04a80000000e800c2
:105fd000b04a8800b04a8000e30f5000020034004d
:105fe0000000eb00b04a8800b54a800025179800f1
:105ff0002e109000e10f500012003200ae10900001
:10600000e18f500004003c002e1190000200e000df
:106010000800320016003700ae119000e28f5100e8
:106020000c0032002e129000e30f52000d003200df
:106030000f003700c14c80006004220019080700df
:106040000b003700c14c8000408821001508070074
:1060500007003700c14c8000e0492100110807000b
:1060600003003700c14c800020f720000d08070016
:1060700040062000600a0700c3c2bf000080fb008a
:106080004400de000080fb00610060000000e000d2
:10609000f9ff320093fc0700aefc0700befc0700ce
:1060a0007809e20002003a00c4e2a90001003700ca
:1060b000c4e2a8007609e20008003200d14c80005a
:1060c000400020000088b900cf80de00c05c88005e
:1060d000d15c88002312070004003700d04c8000f8
:1060e000cf80de00c05c8800d15c88000040eb00ff
:1060f000eb0c0700c5408000151f98001e1890008b
:106100000000e000030032009e189000e18f500074
:10611000dc00320051070700200798002e00900095
:106120000000e000240032002e0090000000e0009b
:1061300004003d00c14c8000e0492100d907070060
:1061400003003700c14c800020f72000d50707006e
:10615000e04a8000a2002000110009000200d800df
:106160008000fd00a00020000088b900e04a8800ff
:10617000ae009000a00020000088b900e24a800034
:1061800000004100e04a8800e04a8000e90f50002a
:1061900002003c00a0002000e04a8800e14a8000a4
:1061a000401f2000808f500002003400401f20005c
:1061b000e04a880081fc0700004b8000e40f50009b
:1061c0000400320014fb070070c0b300e60c0700a7
:1061d000070037007609e20003003a0060162e003f
:1061e000720e070002003700c0c020006f0e0700cb
:1061f000d240800032179800be119000e18f51000c
:106200000b0032003e129000e10f520006003400f5
:10621000be129000e28f5200100032003e1090003b
:10622000e30f50004200320006fb07004100370038
:1062300000172e005d0e07004408e20003003a003c
:1062400040172e00590e07003a00370021002000a9
:10625000204280000d10070036003700a00020000b
:10626000a6f80700cf80de001241800023418000a5
:1062700002014000838148001241880023418800c8
:10628000f06080000000e800f0608800f0608000ae
:10629000ef0f5000270034000000eb00f060880092
:1062a0001041800021418000cc09dd004400de0067
:1062b00000807100c488de00624c80000202b800d9
:1062c000724c80000283b90005017800060141008c
:1062d000634c80000198b9000001410082027800ff
:1062e000340f9800450f98006000b80010418800f6
:1062f000214188003e089000ce089000480add0049
:106300004800de0000007200c808de00004188007e
:10631000a0172e00250e070021002000004180005c
:10632000da0f0700c0172e00200e0700010037000b
:106330000cfb070000c4b300590c07004e08e20034
:106340000c00320092fb070092fa070000c2b30073
:10635000850c070051428000400020000008b80072
:10636000a5942000050040001000be000b0f0700a0
:106370002502370060428000e10f500010003a0013
:1063800083fb0700e0172e00801f7800408020006c
:10639000ebe707008f87e90040802000030e07002d
:1063a00051428000400020000008b800a294200064
:1063b000020040001000be00f80e07001202370075
:1063c000934b8000431798004e129000e10f52004b
:1063d00013003200ce129000e18f520004003c0006
:1063e0004e1090000000e000050032001b00370056
:1063f000ce109000e28f50001100320017003700dd
:1064000063fb07005c09f80050182e00801f78001d
:1064100040802000cae70700e48757000f003700dc
:106420005bfb07005c09f800c0182e00801f780095
:1064300040802000c2e70700e487570007003700cc
:1064400053fb07005c09f80030192e00801f78000c
:1064500040802000bae70700e48757004080200012
:10646000d20d070051428000400020000008b80013
:10647000a2942000020040001000be00c70e0700da
:10648000e1013700e04080006102b9007417980014
:10649000051f9800a0002000010020007e11900040
:1064a0008e199000800f5100818f590012013e001b
:1064b0007e1290008e1a9000046001000a003700de
:1064c0002d0037006100370094003700cd00370001
:1064d00009013700280137004901370067013700fb
:1064e0008e013700aa0137000040eb00ec0b0700db
:1064f000a0192e00ad0d070000c4b300e80b070083
:1065000056060700c14a800000804000c04a88004b
:106510005809e20002003d000000eb00c04a88007c
:10652000c04a8000e20f500002003400200020002a
:10653000c04a8800b01a2e009c0d07005809e200de
:1065400002003a00501b2e00980d0700c04a800040
:10655000e10f500002003a00d01b2e00930d0700ff
:10656000c04a8000e20f5000a7013a00501c2e00e4
:106570008e0d0700a40137000040eb00c80b070098
:1065800055428000551798005e109000e10f5000b2
:106590000e003200de109000e18f500004003c003d
:1065a0005e1190000200e000050032000c00370090
:1065b000de119000e28f5100070032000800370022
:1065c000d01c2e00790d070005003700e01d2e00bd
:1065d000760d070002003700f01e2e00730d070035
:1065e00000c4b300ae0b07001c060700d14a8000b0
:1065f00000804000d04a88005a09e20002003d00b5
:106600000000eb00d04a8800d04a8000e10f500023
:106610000200340010002000d04a8800b01a2e007a
:10662000620d07005a09e20002003a00501b2e00da
:106630005e0d0700d04a8000e10f500072013a0061
:10664000f01f2e00590d07006f0137000040eb00ce
:10665000930b070070202e00540d070000c4b300f8
:106660008f0b0700fd05070020079800ae00900083
:10667000200320000088b900f24a80000000410099
:10668000f04a8800f14a8000007d2000808f500091
:1066900002003400007d2000f04a8800f14a8000aa
:1066a000700c2000808f500002003c00800c200005
:1066b000f04a8800f14a8000800c2000808f500052
:1066c00006003a0080212e00801f780040802000c4
:1066d0001be707008f87e900060037005e09f80016
:1066e00090222e00801f78004080200014e70700d1
:1066f000e4875700408020002c0d070037fb07007f
:106700002e0090000000e0003f013200c14c8000ec
:1067100090428000630607003b0137000040eb0019
:106720005f0b0700b0232e00200d070075f907004e
:1067300000c4b3005a0b0700b04a80000000d0002c
:10674000a496200084044000b04a80000000d000dd
:10675000a596200005044000c005070080007800d1
:10676000a00020000088b900980c4000b04a8000ca
:106770000000d000a2962000820040004077220056
:10678000910f100006003400b04a80000000d000d5
:10679000a396200083004000407722008008780004
:1067a000b04a80000000d000a49620008400400081
:1067b00030062000910f100006003c00b04a800017
:1067c0000000d000a5962000850040004006200073
:1067d0008008780050242e00f40c0700b04a800096
:1067e0000000d000a1962000010040002100200000
:1067f00010007800a50e0700e0242e00eb0c070027
:10680000010137000040eb00250b070030252e006a
:10681000e60c070000c4b300210b07008f0507003a
:10682000014b800000804000004b88006009e200be
:1068300002003d000000eb00004b8800004b800090
:10684000e40f50000200340040002000004b88009c
:10685000024b800062179800ee119000e28f510009
:10686000170032006e129000e20f520007003c0049
:10687000ee1290000500e0000b0032006e10900058
:10688000e10f50000b00320015003700ee109000b1
:10689000e38f50000d0032006e119000e40f5100a4
:1068a0000d0032000e00370040262e00bf0c0700fe
:1068b0000b00370050272e00bc0c070008003700e3
:1068c00060282e00b90c07000500370070292e0043
:1068d000b60c070002003700802a2e00b30c070018
:1068e000004b8000e40f5000c70032000000eb00b6
:1068f000b04b8800c40037000040eb00e80a0700f6
:10690000902b2e00a90c070000c4b300e40a070076
:106910005205070080007800204b800001004000f5
:10692000204b8800214b8000c0442000808f500005
:1069300002003400c0442000204b88006409e200bb
:1069400002003d000000eb00204b88006409f800c5
:10695000a02c2e00801f78004080200078e60700e1
:10696000e487570040802000900c0700204b8000f7
:10697000aa050700a40037000040eb00c80a070082
:10698000c02d2e00890c070000c4b300c40a070004
:106990003205070080007800200320000088b9003d
:1069a000124b800000004100104b8800114b80000a
:1069b000c0da2000808f500002003400c0da2000ce
:1069c000104b88006209e20002003d000000eb006d
:1069d000104b88006209f800d02e2e00801f78002e
:1069e0004080200056e60700e487570040802000e2
:1069f0006e0c0700104b80008e05070082003700e8
:106a00000040eb00a60a0700d02f2e00670c0700fd
:106a100000c4b300a20a070010050700314b800034
:106a200000804000304b88006609e20002003d0013
:106a30000000eb00304b8800304b8000e10f50002d
:106a40000200340010002000304b8800e0302e009f
:106a5000560c07006609e20002003a0060312e0081
:106a6000520c0700304b8000e10f500066003a00e6
:106a700000322e004d0c0700630037000040eb0091
:106a8000870a0700a0322e00480c070000c4b3009c
:106a9000830a0700f1040700500f98005e08900079
:106aa0000000e0000f003200404b8000de08900044
:106ab00001004000404b88006809e20002003d00f0
:106ac0000000eb00404b8800404b8000e70f500077
:106ad0000200340070002000404b8800404b8000d2
:106ae000c2080700414b8000800020000008b80069
:106af00093d92d0000804100801f7800b0332e0014
:106b0000801f7800408020000de60700e4875700d2
:106b100040802000250c07003b0037000040eb00c0
:106b20005f0a070080342e00200c070000c4b30069
:106b30005b0a0700c9040700a14b800000805000d9
:106b4000a04b88007409e20002003d000000eb0049
:106b5000a04b8800a04b8000e10f500002003400e1
:106b600010002000a04b8800b01a2e000f0c070068
:106b70007409e20003003a0090352e000b0c070068
:106b80002100370010362e00080c07001e003700c9
:106b90000040eb00420a070090362e00030c07006d
:106ba00000c4b3003e0a0700ac040700c14b8000dc
:106bb00000804000c04b88007809e20002003d00e0
:106bc0000000eb00c04b8800c04b8000e10f50007c
:106bd0000200340010002000c04b8800b01a2e00c4
:106be000f20b07007809e20002003a00501b2e0069
:106bf000ee0b0700c04b8000e10f500002003a008e
:106c0000f01f2e00e90b0700304b80000000e00071
:106c100002003a00f712070001003700d900070010
:106c2000d4c2bf000080fb0061006000e10f500093
:106c300040fb3a00eaf807003efb37000600fa0086
:106c4000a0372e00801f7800dce507008f87e90061
:106c50000000eb00000f7800f01f20009e0f1000d6
:106c600019003c006401470000002f009e00400016
:106c700013002000f00720004309070010079800c8
:106c80001e0078006f0060000000e00006003a007f
:106c90001e007800801f780010392e00801f7800b9
:106ca000c6e50700e48757002e009000801f78009b
:106cb00090392e00801f7800c0e50700e487570058
:106cc0001e8fe800e4ff37001e009000801f780050
:106cd000e0392e00801f7800b8e50700e4875700f0
:106ce0000080fa00000006000600fa00000f78009d
:106cf0000040eb00204798000000eb0020079800c0
:106d00001e007800801f7800803b2e00801f7800d6
:106d1000aae50700e48757001e00e00018003200d3
:106d2000000f2000801f7800e03d2e00801f7800bb
:106d3000a2e50700e48757002e409000ed4f500079
:106d40000f003200ae009000e00e2000808f500057
:106d50000b003c0066080700204798002e009000ba
:106d60008185200001004000ae409000014878007d
:106d70002e0090000000e80020079800eeff37008a
:106d8000b90d0700f0402e00801f78008be507004a
:106d90008f87e90080852000cf0e07000080fa0071
:106da000000006000200fa000000eb00000f78006f
:106db000f00e20009e0f100006003c008085200091
:106dc0009e0040000040eb00804878001e0fe80065
:106dd000f7ff37000080fa00000006000400fa0008
:106de000000f2000801f780000422e00801f7800d6
:106df00072e50700e4875700eaff07000000eb0098
:106e000010079800d0c0b3009e4f10000e00320053
:106e10009e009000e00e2000808f50000a003c0091
:106e200033080700004f78001e0090008185200085
:106e3000010040001e4878001e0090000000e8009d
:106e400010079800efff370080852000ba0e07007a
:106e500080452e00801f780058e507008f87e900e5
:106e60000080fa00000006000000fa00b0452e0085
:106e7000801f780051e507008f87e900f0472e005a
:106e8000801f78004de507008f87e90080492e00bc
:106e9000801f780049e507008f87e900b04b2e007e
:106ea000801f780045e507008f87e900804d2e00a0
:106eb000801f780041e507008f87e900604f2e00b2
:106ec000801f78003de507008f87e90030512e00d4
:106ed000801f780039e507008f87e900d0522e0027
:106ee000801f780035e507008f87e900d0532e001a
:106ef000801f780031e507008f87e900d0542e000d
:106f0000801f78002de507008f87e90040572e008d
:106f1000801f780029e507008f87e900c0582e0000
:106f2000801f780025e507008f87e900e0592e00d3
:106f3000801f780021e507008f87e900c05a2e00e6
:106f4000801f78001de507008f87e900305c2e0068
:106f5000801f780019e507008f87e900c05d2e00cb
:106f6000801f780015e507008f87e900305f2e004d
:106f7000801f780011e507008f87e9000080fa0084
:106f8000000006001600fa00881f7800b507070009
:106f90000004e000bd013200c2070700204f980046
:106fa0002e4890000081fb0003002000e0fb2f0032
:106fb000f1ff2f000201400083814800120f98006a
:106fc000230f980080032000010020001e0990007c
:106fd000ae099000800f5100818f5900aa013e0038
:106fe0001e089000ae08900000600100f500370018
:106ff000a5013700a4013700a3013700a201370023
:10700000a1013700a0013700650037009e0137005d
:107010009d0137009c0137009b0137009a01370022
:107020009901370098013700970137009601370022
:1070300095013700030137009301370092013700b3
:10704000c7003700900137008f013700f10037008b
:107050008d0137008c0137008b0137008a01370022
:1070600089013700880137007e003700180037009b
:107070008e003700030137008a0037008201370095
:107080008101370080013700450037007e0137005d
:107090007d013700370137007b0137007a01370067
:1070a000190137000d003700360037007601370030
:1070b00025003700150037007301370072013700d3
:1070c0008b003700700137006f013700fd0037007b
:1070d00042ff070037f607006c013700b0602e0052
:1070e000801f7800b5e407008f87e9001af60700d3
:1070f00080852000801f7800e0622e00801f7800cd
:10710000aee40700e48757006001370070632e008b
:10711000801f7800a9e407008f87e9007609e20064
:107120005a013a000000eb00904b8800400020001c
:10713000004b880080852000ff0d07001000200014
:10714000b04b88005101370040652e00801f780049
:107150009ae407008f87e9007609e2004b013a00c4
:1071600010002000904b880040002000004b880059
:1071700080852000f00d07000080eb00b04b8800f8
:1071800042013700a0662e00801f78008be40700c4
:107190008f87e9000000eb00b04b88003b0137000f
:1071a00037f80700000f78009e007800010f980064
:1071b0000e099000e10f5100070032008e09900087
:1071c000e18f51000e0034000e089000e20f5000d5
:1071d000060032000a00370000682e00801f780089
:1071e00076e407008f87e90009003700a06a2e00c7
:1071f000801f780071e407008f87e90004003700e2
:10720000406d2e00801f78006ce407008f87e90036
:10721000b0702e00801f780068e407008f87e900b7
:1072200080d82d00801f780064e407008f87e90074
:10723000f0712e00801f780060e407008f87e9005e
:10724000e0d82d00801f78005ce407008f87e900fc
:1072500030722e00801f780058e407008f87e90005
:107260000a01370090002000000f7800e1002000a4
:107270009e8f100005013c001e0078009ff407005f
:10728000801f78001e017800821f780080742e0015
:10729000801f780049e40700e68757001e0fe800ca
:1072a000f2ff370065fe0700f800370060752e001a
:1072b000801f780041e407008f87e9000000eb00a1
:1072c0002007980012002000010f2f00f007200077
:1072d000ba0707006400470013002000020f2f00c8
:1072e000f1072000d607070054fe0700e70037002b
:1072f00050772e00801f780030e407008f87e90068
:10730000710807002e489000fb4f5000df0032004c
:10731000d40607000004e000fdff3200e10607008c
:10732000204f98002e489000ed4f500001003a0089
:10733000650807002e4890000080fb00801f780041
:10734000807a2e00801f78001ce40700e487570035
:107350002e4890000080fb00ed090700e9ff370090
:10736000407b2e00801f780014e407008f87e9001f
:10737000550807002e489000fb4f5000c300320014
:1073800028070700204f98002e489000ed4f50002e
:1073900001003a004c0807002e4890000080fb00d6
:1073a000801f7800707e2e00801f780003e40700a5
:1073b000e48757002e4890000080fb00d4090700a6
:1073c000ecff3700f07e2e00801f7800fbe3070003
:1073d0008f87e9000000eb00000f7800f005200027
:1073e0009e0f100007003c00370807001e007800c1
:1073f000e1080700200320007f0507001e0fe800ba
:10740000f6ff3700970607000004e000f1ff3200a6
:107410009e00370000802e00801f7800e7e3070001
:107420008f87e9000000eb00000f78002e0090002d
:107430001e017800110009000200d8002007980002
:1074400092003700e0802e00801f7800dbe3070009
:107450008f87e900ae060700000f7800f0832e004a
:10746000801f7800d5e307008f87e900a806070092
:10747000100798009e0090001e0078000903070086
:10748000820037002ef40700104d8000214d80004f
:10749000809fbe0051428000400020000008b800dc
:1074a000c2972000020040001001be00829fbe0073
:1074b00000862e00801f7800c0e30700ea8757008f
:1074c0007200370090872e00801f7800bbe3070012
:1074d0008f87e90086060700204f98002e4890000d
:1074e0000080fb00ef0c07002e4890000080fb009e
:1074f000801f7800a08a2e00801f7800afe307006d
:10750000e487570061003700508b2e00801f780001
:10751000aae307008f87e900514280004000200065
:107520000008b800c3972000030440007806070055
:10753000008cbe0002f40700104d8000214d800039
:10754000809fbe0051428000400020000008b8002b
:10755000c2972000020040001001be00829fbe00c2
:1075600000862e00801f780094e30700ea8757000a
:1075700046003700008d2e00801f78008fe3070043
:107580008f87e900505c8000615c8000809fbe00b6
:10759000608e2e00801f780088e30700e687570082
:1075a000e25c8000f35c8000829fbe00b08f2e0002
:1075b000801f780081e30700e6875700c05c8000e9
:1075c000d15c8000809fbe0000912e00801f78005b
:1075d0007ae30700e6875700a00bf80050922e00d0
:1075e000801f780075e30700e48757005408f8000f
:1075f00090932e00801f780070e30700e487570007
:107600005608f800d0942e00801f78006be3070026
:10761000e4875700c4c2bf000080fb004600de00c4
:107620000080fb0061006000801f7800cac2bf00bc
:107630000080fb004200de000080fb006100600073
:10764000801f7800e8c2bf000080fb004200de001f
:107650000080fb0061006000801f7800e9c2bf006d
:107660000080fb004400de000080fb006100600041
:10767000801f780010962e00801f78004fe30700cf
:10768000ea87570001003700f7fd07004f04780034
:107690000080fa00000006001c00fa00889fbe006f
:1076a000a7f30700b5f307003f0707000000eb0052
:1076b0002207070041f7070048f707000000eb002a
:1076c000000f78008007070030002000b0428800db
:1076d00010002000a0428800304b8000e10f5000d5
:1076e00008003a0080982e00801f780033e30700de
:1076f0008f87e900509a2e00801f78002fe3070043
:107700008f87e90000000000e8c2bf000080fb0096
:107710004200de000080fb00610060000000e0002d
:107720000300320010002000604288000200370091
:107730000000eb006042880032f7070062f60700a5
:10774000d00020006df3070040418800c0002000f9
:107750006af30700504188004141800040418000a9
:107760000088b900a0418800b141880051418000e3
:10777000504180000088b900c0418800d141880094
:10778000a2418000b3418000c0418000d14180000f
:107790000000510081805900e0418800f1418800db
:1077a000d0f60700ebf60700fbf60700c3c2bf00e8
:1077b0000080fb004500de000080fb0061006000ef
:1077c0000000e00013003a001e0fe80060002000f7
:1077d0009e0f1000020034000000eb00000f780044
:1077e00021032000e02521002e020700c3c2bf00b4
:1077f0000080fb004500de000080fb0061006000af
:107800000000e000f9ff3200400620007a04070083
:10781000920107009e007800510f98005e099000c9
:10782000e30f5100a8003200de099000e38f510001
:1078300007003c005e0a9000e10f52003400320065
:10784000de0a9000e18f52007b003c000900370007
:107850005e089000e50f5000fc003200de0890004a
:10786000e48f5000c90034005e099000e60f51001b
:10787000140132000040eb0009070700309d2e0084
:10788000ca08070000c4b300050707005142800082
:10789000400020000008b800c39720008304400087
:1078a00051428000400020000008b800c49720002a
:1078b000040440006901070080007800a000200057
:1078c0000088b900cf80de00b81c4000a8944800b2
:1078d0006601470051428000400020000008b800c7
:1078e000c5972000050040001002be00849fbe0026
:1078f000409e2e00801f78000200780090e2070072
:10790000e687570066004700a8080700f500370023
:107910000040eb00e2060700a0002000f7f207009d
:10792000cf80de00624c80000202b800724c800002
:107930000283b9000501780006014100634c800014
:107940000198b900000141008202780014079800f4
:10795000250798001e009000ae009000c80add00c8
:107960004800de0000807200c808de000041880088
:10797000109f2e008d08070021002000004180008c
:10798000420a0700a09f2e008808070000c4b30029
:10799000c306070031010700cf80de00624c800083
:1079a000734c80000201400083814800624c8800d3
:1079b000734c8800624c8000734c800030062000bd
:1079c00001002000800f5100818f590004003c000d
:1079d0004006200001002000604c8800714c8800a7
:1079e000624c8000734c8000800c2000010020005d
:1079f000800f5100818f590004003400800c20005a
:107a000001002000604c8800714c8800660047002f
:107a1000644c8000754c8000849fbe00e19f2e0066
:107a2000811f780046e20700e6875700660047009e
:107a30005e080700ab0037000040eb009806070027
:107a4000e600470010a12e00801f7800010078009a
:107a50003be207008f87e9006600470053080700f4
:107a600000c4b3008e060700fc0007008000780009
:107a7000c04c800001004000c04c88009809e20022
:107a800002003d000000eb00c04c8800c14c8000ab
:107a900040062000808f5000020034004006200085
:107aa000c04c8800660047009809f80021a22e000b
:107ab000811f780022e20700e48757006600470034
:107ac0003a080700870037000040eb007406070003
:107ad00030a32e0035080700daf4070000c4b30015
:107ae0006f060700dd000700cf80de00a24c80009b
:107af000b34c80000201400083814800a24c880002
:107b0000b34c8800a04c8000b14c8000e00f5000c6
:107b1000e08f580003003d006000b800a04c8800d2
:107b2000b14c8800a24c8000b34c8000400620007d
:107b300001002000800f5100818f590004003400a3
:107b40004006200001002000a04c8800b14c8800b5
:107b5000a44c8000b54c8000844c8800954c880073
:107b600066004700a24c8000b34c8000829fbe009c
:107b7000e19f2e00811f7800f1e10700e6875700a2
:107b80006600470009080700560037000040eb0078
:107b900043060700c0a32e0004080700f1f4070005
:107ba00000c4b3003e060700ac000700cf80de0033
:107bb000444c8000554c80000402400085824800ff
:107bc000444c8800554c8800424c8000534c800047
:107bd00070bb200001002000800f5100818f5900f0
:107be00004003c0080bb200001002000404c8800c5
:107bf000514c8800424c8000534c8000803821005a
:107c000001002000800f5100818f590004003400d2
:107c10008038210001002000404c8800514c880031
:107c200066004700424c8000534c8000829fbe009b
:107c300061a42e00811f7800c1e10700e68757008c
:107c400066004700d9070700260037000040eb0018
:107c50001306070070a52e00d407070000c4b30068
:107c60000f0607007d00070080007800d04c8000e0
:107c700001004000d04c8800d04c8000e40f500040
:107c800002003c0050002000d04c8800d04c800006
:107c9000ea0f500002003400a0002000d04c880001
:107ca000660047009a09f80081a62e00811f78001f
:107cb000a3e10700e487570066004700bb07070001
:107cc000080037000040eb00f5050700b0a72e00c4
:107cd000b607070000c4b300f1050700c0a82e00d6
:107ce000b2070700630020009e8f110031003a00a8
:107cf000cec2bf000080fb004400de000080fb001d
:107d0000610060000000e0004a003a00803e200070
:107d1000305d8800cec2bf000080fb004400de0062
:107d20000080fb00610060000000e00041003a00bc
:107d3000a60be200f7ff3a003df30700acf20700a4
:107d40004cf20700c14c8000a00020000088b90060
:107d500080007800c0f62000d20007000000eb0091
:107d6000f0408800d8050700d0a92e008f07070033
:107d7000304b8000e10f500004003a00e0aa2e00d2
:107d8000801f78008de107008f87e900c05d20002b
:107d900019030700cec2bf000080fb004400de00d4
:107da0000080fb00610060000000e000f9ff32008d
:107db00027003700cec2bf000080fb004400de0079
:107dc0000080fb00610060000000e00019003a0044
:107dd00087f20700c14c8000c0f62000b100070008
:107de0000000eb00f0408800b7050700a0ac2e00b3
:107df0006e070700304b8000e10f500004003a008e
:107e000080ad2e00801f78006ce107008f87e900ad
:107e100000000000cec2bf000080fb004400de0076
:107e20000080fb00610060000000e000f9ff32000c
:107e300007003700d4c2bf000080fb006100600073
:107e4000e10f500030fe3a0065f407002efe3700c7
:107e50004f04be000080fa00000006000200fa0095
:107e6000d05d8000000f78000000eb00d05d88003e
:107e70001e0078000080fa00000006000000fa00f2
:107e80007409e2000a003a00960be2000400320096
:107e9000e982a800e842a800e862a80012003700c2
:107ea000e982a900e842a900e862a9000e003700b3
:107eb000c8c2bf000080fb004300de000080fb0062
:107ec000610060000000e00004003200e982a800c8
:107ed000e842a800e862a80003003700e982a90090
:107ee000e842a900e862a9000080fa00000006004c
:107ef0000000fa0010002000b05c8800f04c800008
:107f0000014d80000d050700ca42a800c4c2a800a8
:107f10000080fa00000006000000fa00f04c80002b
:107f2000014d800005050700ca42a800c4c2a80090
:107f30000080fa00000006000000fa00c4c2a90098
:107f4000ca42a9006000b800fc0407000000eb0072
:107f5000b05c8800580ce20006003200b06280007d
:107f6000904b8800a0628000004b88000000eb006e
:107f7000c06288000080fa00000006000000fa00dd
:107f8000d04c8000cf80de00c05c8800d15c8800cf
:107f90000000eb00b05c8800803e2000305c880070
:107fa0000000eb00800c88000000eb00b00c8800a3
:107fb00040062000600c880040062000700c8800fd
:107fc000e0002000800c8800007d2000900c8800dc
:107fd000007d2000a00c8800e0002000b00c88008c
:107fe000b0cc21007008880013e1a8008ce0a80044
:107ff000d222a90020002000300c880020002000a0
:10800000400c880060002000500c880011e1a9009d
:108010008cc0a9000080fa00000006000200fa00ef
:10802000000f78001e007800600c88000080fa00c5
:10803000000006000200fa00000f78001e00780021
:10804000900c88000080fa00000006000200fa0090
:10805000000f7800301724009e0f10000b003c002a
:108060000000eb00300888001e0078000000d000ff
:108070000000e900600888001e007800300c8800cd
:108080001e007800400c880011e1a8000080fa0072
:10809000000006000000fa0011e1a9000080fa00cb
:1080a000000006000400fa00000f78001107980095
:1080b000505c8000615c8000e00f5000e08f580051
:1080c00007003a001e0090000000e00004003400a9
:1080d0001e009000405c88001e007800dbff070057
:1080e0000080fa00000006000000fa000000eb002b
:1080f000805c88005408e20010003200005d8000bf
:10810000cf80de00c25c80000012b800c25c80003c
:108110000193b9000501780006014100d35c80009d
:108120000380b9000001410082027800e45c88000d
:10813000f55c88006eff07000f003700005d8000cf
:10814000cf80de00c25c80000012b800c25c8000fc
:108150000193b9000501780006014100d35c80005d
:108160000380b9000001410082027800e45c8800cd
:10817000f55c880068ff0700f14a8000800c200051
:10818000808f500004003200015d8000904280002a
:10819000c4ff070003003700015d80000000eb0012
:1081a000c0ff0700005d80000000d000cf80de002f
:1081b000505c8800615c88000080fa0000000600c6
:1081c0000000fa0010002000805c88005408e200e3
:1081d00010003200005d8000cf80de00c25c8000b5
:1081e0000012b800c25c80000193b900050178005c
:1081f00006014100d35c80000380b900000141000a
:1082000082027800e45c8800f55c880038ff070093
:108210000f003700005d8000cf80de00c25c800070
:108220000012b800c25c80000193b900050178001b
:1082300006014100d35c80000380b90000014100c9
:1082400082027800e45c8800f55c880032ff070059
:10825000f14a8000800c2000808f5000070032001f
:10826000015d8000300020000088b90080007800a7
:10827000904280008bff070006003700015d800000
:10828000300020000088b900800078000000eb007a
:1082900084ff0700015d8000400020000088b900d5
:1082a000cf80de00505c8800615c88000080fa00ae
:1082b000000006003600f800809fbe00829fbe00ce
:1082c000849fbe00869fbe000400fa0084e0a900df
:1082d000ca02a800880be20007003200405c800060
:1082e0000000e900405c8800880be20002003a00d0
:1082f00068ff0700c4c2a900e05c8000f15c800058
:10830000e00f5000e08f58000c003200e05c80006d
:10831000f15c800061005000e0805800e05c880063
:10832000f15c8800e05c8000f15c8000e00f5000b0
:10833000e08f580001003a00fffe0700505c80000b
:10834000615c8000e00f5000e08f580012003200a6
:10835000505c8000615c800061005000e08058004b
:10836000505c8800615c8800505c8000615c80002b
:10837000e00f5000e08f580007003a00900be20039
:1083800003003a0010002000905c880002003700d3
:1083900010002000a05c8800a0080700b042800008
:1083a000e20f500011003a00e1c2bf000080fb0064
:1083b000610060000000e00002003a000000eb00f5
:1083c000905c8800e0c2bf000080fb004600de0039
:1083d0000080fb00610060000000e00019003a002e
:1083e0000000eb00a05c880016003700e1c2bf006f
:1083f0000080fb00610060000000e00003003a0024
:108400000000eb00905c88000200370010002000a4
:10841000905c8800e0c2bf000080fb004600de00e8
:108420000080fb00610060000000e00003003a00f3
:108430000000eb00a05c8800020037001000200064
:10844000a05c8800b1428000110798001e009000d7
:10845000e20f500007003c009e0090000100e00089
:1084600022003c001e0090000000e00005003200e9
:108470007f0037009e009000e38f500041003200e3
:108480007b003700e1c2bf000080fb00610060009c
:108490000000e00007003a00505c8000615c800052
:1084a000e00f5000e08f580002003a000eff070076
:1084b0006f003700e0c2bf000080fb004600de0016
:1084c0000080fb00610060000000e00068003a00ee
:1084d000505c8000615c8000e00f5000e08f58002d
:1084e00063003a0036ff070061003700900be2009e
:1084f00012003200920be20007003a00505c80004c
:10850000615c8000e00f5000e08f580002003a00ec
:10851000f5fe070056003700940be20054003a00c5
:10852000505c8000615c8000e00f5000e08f5800dc
:108530004f003a0022ff07004d003700940be20085
:1085400007003a00505c8000615c8000e00f500042
:10855000e08f580002003a0019ff0700440037007e
:10856000920be20042003a00505c8000615c8000a7
:10857000e00f5000e08f58003d003a00dafe07009f
:108580003b003700e1c2bf000080fb0061006000db
:108590000000e0002b003a008e0be20008003a00d9
:1085a00010002000705c8800f14a8000800c2000e0
:1085b000808f50000200320090428000a3fe07002e
:1085c0005408e20010003200005d8000cf80de0021
:1085d000c25c80000012b800c25c80000193b90048
:1085e0000501780006014100d35c80000380b900da
:1085f0000001410082027800e45c8800f55c88009c
:108600003bfe07000f003700005d8000cf80de00da
:10861000c25c80000012b800c25c80000193b90007
:108620000501780006014100d35c80000380b90099
:108630000001410082027800e45c8800f55c88005b
:1086400035fe0700e1c2bf000080fb006100600052
:108650000000e000060032008e0be2000400320051
:10866000c4c2a9008bfe07000000eb00705c88000c
:1086700002fe0700a60be20003003200305d80001e
:108680000000e900305d8800305c80000000e900f7
:10869000305c8800860be20005003a00803e200036
:1086a000305c8800104080000000e8001040880026
:1086b000205c80000000e900205c8800840be20060
:1086c00009003d00401f2000205c8800a40be20050
:1086d00003003a0010002000205d880002003700ef
:1086e0000000eb00205d8800a80be20003003200d0
:1086f000405d80000000e900405d8800820be200e0
:1087000003003200105c80000000e900105c88006b
:10871000505d80000000d000505d8800c3c2bf00e3
:108720000080fb004700de000080fb000000e0004e
:1087300004003a00505d80000000a000505d8800f9
:1087400004003700505d8000e1ff2f000100600051
:10875000505d8800605d80000000d000605d880092
:10876000c3c2bf000080fb004600de000080fb00ab
:10877000610060000000e00004003a00605d8000dd
:108780000000a000605d880004003700605d80008c
:10879000e1ff2f0001006000605d8800ae0be20089
:1087a0000b003a00505d8000e10f400010003a00dd
:1087b00010002000705d8800401f2000b05d880020
:1087c000d05d80000000e800d05d88000800370020
:1087d000aa0be20006003a000000eb00705d880082
:1087e0000000eb00b05d88000000eb00905d8800a9
:1087f000b00be2000b003a00605d8000e10f40002a
:1088000010003a0010002000805d8800401f20000a
:10881000c05d8800d05d80000000e900d05d880068
:1088200008003700ac0be20006003a000000eb0045
:10883000805d88000000eb00c05d88000000eb0058
:10884000a05d8800b60be20007003200b05d80003a
:108850000000e900b05d8800b60be20002003a00bb
:1088600000052000905d8800b80be2000700320090
:10887000c05d80000000e900c05d8800b80be20028
:1088800002003a0000052000a05d8800b20be20063
:108890000a003200905d80000000e900905d8800d1
:1088a000b20be20005003a0000052000905d880050
:1088b000d05d80000000e800d05d8800b40be200cd
:1088c0000a003200a05d80000000e900a05d880081
:1088d000b40be20005003a0000052000a05d88000e
:1088e000d05d80000000e900d05d8800bc0be20094
:1088f00003003200e05d80000000e900e05d8800d8
:10890000be0be20003003200f05d80000000e900d1
:10891000f05d8800105d80000000e800105d8800b8
:10892000ca02a9000080fa004f03be004f02be0039
:108930004f01be004f00be003600f90000400600a7
:108940000200fa00000f78000000eb00c008880069
:108950001e00780001002000820020000202b80002
:108960000001eb000283b900050178000601410017
:10897000830020000388b9000001410082027800d2
:10898000e408880086c0a90021e1a80086c0bf00d5
:108990000080fb004600de000080fb0061006000fc
:1089a0000000e000f9ff320021e1a9000080fa0098
:1089b000000006000000fa000000eb00c00888007c
:1089c000c0cc2100e008880086c0a90021e1a800f1
:1089d00086c0bf000080fb004600de000080fb0078
:1089e000610060000000e000f9ff320021e1a90011
:1089f0000080fa00000006000400fa00000f780072
:108a00000000eb00100798001e0090009e0f500021
:108a100005003100e7ff07001e0090000000e8009d
:108a200010079800f8ff37000080fa0000000600e9
:108a30003600f800809fbe00829fbe00849fbe006b
:108a4000869fbe000200fa0030032000a0108800bc
:108a50000000eb00000f7800f0cf27009e0f100001
:108a600003003c00000000001e0fe800faff370082
:108a700000b02e00801f780050de07008f87e900cd
:108a80004207f800a0b12e00801f78004bde0700df
:108a9000e48757009a000700ffff37003600f80010
:108aa000809fbe00829fbe00849fbe00869fbe0046
:108ab0000000fa00105f8800215f8800325f8800a4
:108ac000435f8800545f8800655f8800765f880098
:108ad000875f8800985f8800a95f8800ba5f880078
:108ae000cb5f8800dc5f8800ed5f8800fe5f880058
:108af0000f60880080b22e00801f78002fde0700f4
:108b00008f87e900e20bf80000b42e00801f780088
:108b10002ade0700e4875700e40bf800a0b42e001b
:108b2000801f780025de0700e4875700e60bf80079
:108b300040b52e00801f780020de0700e487570034
:108b4000e80bf800e0b52e00801f78001bde070060
:108b5000e4875700ea0bf80080b62e00801f7800eb
:108b600016de0700e4875700ec0bf80020b72e0054
:108b7000801f780011de0700e4875700ee0bf80035
:108b8000c0b72e00801f78000cde0700e487570076
:108b9000f00bf80060b82e00801f780007de070099
:108ba000e4875700f20bf80000b92e00801f780010
:108bb00002de0700e4875700f40bf800a0b92e008e
:108bc000801f7800fddd0700e4875700f60bf800f2
:108bd00040ba2e00801f7800f8dd0700e4875700b8
:108be000f80bf800f0ba2e00801f7800f3dd0700c4
:108bf000e4875700fa0bf800a0bb2e00801f780016
:108c0000eedd0700e4875700fc0bf80050bc2e0097
:108c1000801f7800e9dd0700e4875700fe0bf800ad
:108c200000bd2e00801f7800e4dd0700e4875700b8
:108c3000000cf800b0bd2e00801f7800dfdd0700bb
:108c4000e48757002e000700ffff37003600f800ca
:108c5000809fbe00829fbe00849fbe00869fbe0094
:108c60000000fa000f6088000f90200060be2e0008
:108c7000801f7800d1dd07008f87e900000cf80025
:108c8000b0bd2e00801f7800ccdd0700e4875700c0
:108c90001b000700ffff37003600f800809fbe0072
:108ca000829fbe00849fbe00869fbe000000fa0027
:108cb000c0bf2e00801f7800c0dd07008f87e9004d
:108cc0000f000700ffff37003600f800809fbe004e
:108cd000829fbe00849fbe00869fbe000000fa00f7
:108ce00090a0a9009120a90010c12e00801f78003b
:108cf000b2dd07008f87e90001000700ffff3700a2
:108d00000000fa00f0010700e0c22e00a7030700f0
:108d1000d4c2bf000080fb0061006000e10f500082
:108d2000fbff3a00cfa2a900f9ff3700809fbe00e9
:108d3000829fbe000400fa0090108000004f78006f
:108d400064ccbf000040e80020479800ae4090008f
:108d5000a6c9bf00000ce1000900320042c6200095
:108d600092407800014078000080fb00739a200058
:108d7000030040001e4878008140e8000149780067
:108d80000ec2bf000080fb000000d1000080fb008d
:108d900061006000e10f500001003a000e22a900be
:108da0008520a9000080fa004f01be004f00be00e0
:108db000004006000000fa0000c42e0030009000c1
:108dc000a01088000000eb00601088000000eb009d
:108dd000701088008520a9008d20a8000de2a80051
:108de0000f42a8000080fa00000006000200fa000e
:108df000000f7800700020009e0f10000200340069
:108e000070002000000f780001c42e001e007800c2
:108e10000000d0000100400010007800a010880081
:108e20000080fa00000006000200fa00004f7800ff
:108e30000fc2bf000080fb000000d1000080fb00db
:108e400061006000e10f5000f9ff32001e00fb00de
:108e5000f10f200001006000801088000080fa00ff
:108e6000000006000000fa0041c620009140780092
:108e7000a6c9bf0000c050000040e9000080fb0010
:108e80000080fa00000006000000fa000040eb003d
:108e9000a6e9b70010c0b30064ecb7000080fa0088
:108ea000000006000200fa0000000000a6c9bf0092
:108eb0000040e800004f78009e40780064ccbf007e
:108ec000000ce100f9ff3200a6c9bf000040e80035
:108ed000a6e9b700a6c9bf000080fb00719a200078
:108ee000010040001080fb000080fa000000060036
:108ef0000200fa00ebff0700004f78001e407800e8
:108f0000c9ff07001e80fb000080fa000000060079
:108f10000600fa006000b800008fbe00e1ff070005
:108f20000074a100404798004e409000beff07002b
:108f3000ce409000f0c2b30080cf50001600340045
:108f4000ce40900090c3b30080cf500012003c0090
:108f50001e00be00a20020000203b8000001eb00ca
:108f60000282b9000701780004014100a30020003b
:108f70000388b90000014100820378004e40900050
:108f80000000fb0001fd2f0001004000cf80de004b
:108f9000001f430001974b004e409000ed4f5000e2
:108fa000deff3a001e00be000080fa00000006004e
:108fb0000400fa00004f780090c3b3009e4f1000e9
:108fc00005003e0000cdb3001e4040000000fb0045
:108fd000100798001000370060c4b3009e4f1000c7
:108fe00005003e0090ccb3001e4040000000fb0096
:108ff000100798000800370060c6b3009e4f1000ad
:1090000005003e0090cab3001e4040000000fb0077
:1090100010079800000037001e0090000080fa0042
:10902000000006000400fa009eff07002047980099
:109030002e4090007cff07002e409000dcff0700d0
:10904000104798001e409000004f780095ff0700e1
:10905000204798002e40900073ff07002e4090009c
:10906000d3ff0700104798009e80fb0000012000fe
:109070000088b900804078001e40900000cf40007a
:109080001e80fb000080fa00000006000600fa00c7
:10909000881f7800008fbe0090c0b3005047980032
:1090a0000040eb00404798004e409000e94f5000d0
:1090b00016003c005e4090000000fb0071aa2000fa
:1090c000010440001e00be00a2002000030020009a
:1090d000b1e8070002c3b300024c40001e00be000e
:1090e000a2002000030020009be80700008fbe00c4
:1090f0005e4090000040e900504798004e409000cc
:109100000040e80040479800e7ff37000040eb00d0
:10911000b1eab7004f0478000080fa0000000600b2
:109120000400fa00008fbe001e00be00d7ff07003b
:10913000a7cabf003cff0700a8cabf003aff07004c
:10914000a9cabf0038ff0700aacabf0036ff070040
:10915000abcabf0034ff0700accabf0032ff070034
:10916000adcabf0030ff0700aecabf002eff070028
:10917000afcabf002cff0700b0cabf002aff07001c
:109180000080fa00000006003200f800900188001c
:109190006118e100040032007018e10002003200a2
:1091a000f0ff2f00030037003119ba008301e900f6
:1091b000fdff3a003200f90000000600849fbe0067
:1091c0004220a900440424006110e1000a0032009a
:1091d000540424007010e1000700320064042400ed
:1091e000f5ff2f000510e10003003200f0ff2f0013
:1091f0004f02be00000006003200f800203b88004d
:10920000113b8800043b88000500fc00500520004d
:10921000303b8800a00a2000303b880061e7a800ae
:10922000000000000000000061e7af00feff370013
:109230000000eb003200f9004f02be000000060003
:10924000841f78004220a900440024006118e10036
:1092500006003200540024007018e10003003200c0
:109260004f027800f0ff2f00000006003200f800e7
:1092700091018800821f78003019bb008301e9004a
:10928000fdff3a00213b88004f017800123b880027
:10929000043b88000500fc0050052000303b88009e
:1092a000a00a2000303b880061e7a8000000000011
:1092b0000000000061e7af00feff37000000eb0098
:1092c0003200f9004f027800000006000400fa00a6
:1092d000000f7800cae2a800ca82a800cae2a9006a
:1092e0000040eb00204798002e409000ef4f5000c8
:1092f0000f003c001e00e00002003500cac2a900b9
:1093000001003700cac2a800ca82a90000000000fc
:10931000ca82a8001e0078000000d000000f78006c
:109320002e4090000040e80020479800eeff3700f4
:10933000cae2a8000080fa00000006000600fa0059
:10934000008fbe001e00be004209dd004e00de00a0
:1093500000007100ce08de00f2ff23000200600072
:109360002007980000002100d8ff0700ae00900001
:109370000000240000807000d4ff0700f0ff2300ed
:109380001e006000200798000000eb00cfff0700e0
:10939000ae0090000000240000807000cbff0700aa
:1093a0000080fa00000006000000fa000010200013
:1093b000c6ff070000002c00c4ff07006000b800d3
:1093c000deff07000080fa00000006000200fa003d
:1093d000004f78000900fc00b1168000f00f20005b
:1093e000008160001e80fb00c800dd0000f02f003f
:1093f0000080600000007100b0168800100020009e
:109400004ffd0700d6a2a800100020004cfd070069
:10941000d6a2a9001000200049fd07000080fa0034
:10942000000006000200fa0000002800000f78008b
:109430000400fc009116800000f02f0000807000f6
:1094400090168800d6c2a800d6e2a9001e00e0004f
:109450000a003d001000200039fd0700d6a2a80038
:109460002000200036fd0700a116800000f02f002c
:10947000008f6000d6a2a900f4ff3700d6c2a90071
:10948000d6e2a8000400fc0090168000f10f200036
:1094900001006000901688000080fa0000000600bd
:1094a0000200fa00004f7800deff0700d6e2a900b4
:1094b00000c8b3001e407000c4ff0700d6e2a80039
:1094c0000080fa00000006000000fa00d5ff070047
:1094d000d6e2a90010c0b300bcff0700d6e2a80086
:1094e0000080fa00000006000000fa00d6e2a900a1
:1094f000d6c2a900f00020003ffd070080c3b300e2
:10950000b2ff0700500020003bfd070080c3b300fe
:10951000aeff07001000200037fd070080c3b30036
:10952000aaff07001000200033fd0700c0c0b300f1
:10953000a6ff0700100020002ffd070010c0b30099
:10954000a2ff0700200020002bfd070060c0b30031
:109550009eff07001000200027fd0700d6e2a800ac
:109560000080fa00000006000200fa00004f7800b8
:10957000acff07001e40780094ff07000080fa004f
:10958000000006000200fa00004f78001147980022
:10959000a4ff0700d6e2a900f0c3b3001e4f60008d
:1095a00000c4b3001e40700088ff0700d6e2a80088
:1095b0009cff07001e40900084ff0700c2ff0700c9
:1095c0000080fa00000006000400fa00004f780056
:1095d000114798000040eb0020479800ae409000f3
:1095e0001e40900080cf500007003d008dff070017
:1095f0001e40780075ff07002e4090000040e800f4
:1096000020479800f5ff37000080fa0000000600b0
:109610000000fa0083ff0700d6e2a90000c4b300ef
:109620006aff0700d6e2a80011c0b3000040eb00bb
:10963000e5ff070051c0b30000c1b300e2ff07001f
:1096400021c0b3000040eb00dfff070011c0b300f2
:109650000040eb00dcff070051c0b30040c1b30085
:10966000d9ff070021c0b3000040eb00d6ff070080
:1096700011c0b3000040eb00d3ff070051c0b3009e
:1096800050c1b300d0ff070021c0b3000040eb0081
:10969000cdff070011c0b3000040eb00caff070078
:1096a00051c0b30010c0b300c7ff070021c0b30012
:1096b0000040eb00c4ff070011c0b300c0c1b300fd
:1096c000c1ff070011c0b30040c1b300beff0700d7
:1096d00011c0b300c0c1b300bbff070051c0b3004d
:1096e0000040eb00b8ff070021c0b3000040eb00d2
:1096f000b5ff070011c0b30000c1b300b2ff0700ff
:1097000011c0b3000040eb00afff070011c0b30071
:1097100000c1b300acff070031c0b3000040eb0054
:10972000a9ff070031c0b3000040eb00a6ff07000f
:1097300011c0b30000c1b300a3ff070041c0b300d4
:109740000040eb00a0ff070021c0b3000040eb0089
:109750009dff070031c0b30000c1b3009aff0700ae
:1097600031c0b3000040eb0097ff070056ff070031
:109770000080fa00000006001200fa00000f7800d6
:10978000000320009e0f10000200340000032000a0
:10979000000f78001e007800620020001100090010
:1097a0000200d800200798001e0078006200200008
:1097b000110009000200d8008000fd003007980069
:1097c0000000eb00400798000000eb001007980035
:1097d0001e009000e70f50000e003c00ea0047001a
:1097e0004e00900000814000c1c52e001e00900078
:1097f00000804000104978004e0090000000e80012
:10980000400798001e0090000000e8001007980034
:10981000efff37000000eb00400798002e0090009b
:109820000000e0000c003400ea0047004e00900009
:109830008080400020c0b300804878004e00900037
:109840000000e800400798002e0090000000e900aa
:1098500020079800f1ff37003e0090000000e00074
:1098600007003400ea0047004e00900000814000ed
:1098700001c52e003e009000008040001049780095
:109880000000eb00100798001e009000e70f50004a
:1098900009003c00ea0047001e00900000804000e4
:1098a0001040780030ff07001e0090000000e80024
:1098b00010079800f4ff37000080fa00000006004f
:1098c0001600fa00000f780011079800000320002e
:1098d0009e0f10000200340000032000000f7800eb
:1098e00080002000500798001e00780062002000d1
:1098f000110009000200d800300798001e0078000f
:1099000062002000110009000200d8008000fd0064
:10991000400798001e0090000000e00036003a006a
:109920000000eb00600798003e0090000000e0009f
:109930000f003400ee0047006e0090008080400071
:1099400020c0b300804878006e0090000000e8005e
:10995000600798003e0090000000e9003007980082
:109960005e0090000000e90050079800eeff37000d
:109970004e0090000000e0000d003400ee004700b3
:109980006e0090000081400001c52e004e00900046
:1099900000804000104978006e0090000000e80050
:1099a000600798005e0090000000e90050079800f2
:1099b0000000eb0020079800ae0090005e009000d1
:1099c000808f500042003d00ee0047006e00900086
:1099d0008080400000c2b300804878006e00900094
:1099e0000000e800600798002e0090000000e800ea
:1099f00020079800f0ff37007000200060079800f3
:109a00003e0090000000e0000f003400ee00470030
:109a10006e0090008080400020c0b3008048780035
:109a20006e0090000000e900600798003e00900082
:109a30000000e900300798005e0090000000e90097
:109a400050079800eeff37004e0090000000e00045
:109a50000d003400ee0047006e00900000814000d1
:109a600061c52e004e009000008040001049780033
:109a70006e0090000000e900600798005e00900012
:109a80000000e900500798000000eb002007980054
:109a9000ae0090005e009000808f50000c003d00f2
:109aa000ee0047006e0090008080400000c2b300ce
:109ab000804878006e0090000000e9006007980080
:109ac0002e0090000000e80020079800f0ff37000b
:109ad0000000eb00200798002e009000e70f5000d8
:109ae00009003c00ee0047002e009000008040007e
:109af000104078009cfe07002e0090000000e80057
:109b000020079800f4ff37000080fa0000000600ec
:109b10000200fa00004f78001e40780092fe070015
:109b20000080fa00000006000200fa00004f7800f2
:109b30001e407800104798001e80fb004400de00a5
:109b4000004f780090c0b3009e4f100003003e000d
:109b500000c3b3001e4f40000200370070c3b300c3
:109b60001e4f40001e4078007ffe07001e40900000
:109b7000004f78001e4078006f4f600090c0b30027
:109b80009e4f100003003e0000c3b3001e4f400074
:109b90000200370070c3b3001e4f40001e40780023
:109ba00071fe07000080fa00000006000200fa00c3
:109bb000000f78001e0078001004e000070032005b
:109bc0009e0078001140780067fe07001e007800b4
:109bd0000000e800000f7800f6ff37000080fa0070
:109be000000006000600fa00008fbe004247980001
:109bf0004e4090000004e0002e003a001e00be001f
:109c000002a02c00a3b92300c4e507000043b00064
:109c100055fe07001e00be0002a02c00a3b92300c1
:109c2000bee5070002a02c000202b800a2b9230082
:109c30000283b900050178000601410003a02c0051
:109c40000388b90000014100820278001e1f120043
:109c50001e971a00e0c2b30043fe07001e00be00bc
:109c600002102e00535f2000ace507000043b00057
:109c70003dfe07001e00be0002102e00535f2000b4
:109c8000a6e5070002102e000202b800525f200075
:109c90000283b900050178000601410003102e007f
:109ca0000388b90000014100820278001e1f1200e3
:109cb0001e971a004e4090000004e0000a00320097
:109cc0001e00be00026829008309200093e50700fa
:109cd000e00f5000e08f580003003a0000c2b300cc
:109ce00021fe0700060037001e00be0002682900a2
:109cf0008309200089e507000043b0001afe070031
:109d00001e00be00026829008309200083e50700c9
:109d1000026829000202b800820920000283b9000b
:109d20000501780006014100036829000388b90095
:109d300000014100820278001e1f12001e971a00c7
:109d40001e00be0002242400f300200073e507007b
:109d50000043b00004fe07001e00be0002242400e1
:109d6000f30020006de50700022424000202b80081
:109d7000f20020000283b9000501780006014100cd
:109d8000032424000388b900000141008202780006
:109d90001e1f12001e971a00e0c2b300f2fd07005a
:109da0001e00be00026a2800130020005be50700c9
:109db0000043b000ecfd07001e00be00026a280050
:109dc0001300200055e50700026a28000202b800cf
:109dd000120020000283b90005017800060141004d
:109de000036a28000388b90000014100820278005c
:109df0001e1f12001e971a001e00be0002712200d4
:109e00000300200045e507000043b000d6fd070031
:109e10001e00be0002712200030020003fe5070083
:109e2000027122000202b8000001eb000283b900b7
:109e30000501780006014100037122000388b90082
:109e400000014100820278001e1f12001e971a00b6
:109e50001e00be00823e2000030020002fe5070008
:109e60000043b000c0fd07001e00be00823e20007f
:109e70000300200029e50700823e20000202b8000e
:109e80000001eb000283b9000501780006014100e2
:109e9000833e20000388b90000014100820278005f
:109ea0001e1f12001e971a00e0c2b300aefd07008d
:109eb0001e00be00420620000300200017e5070038
:109ec0000043b000a8fd07001e00be0042062000af
:109ed0000300200011e50700420620000202b8003e
:109ee0000001eb000283b900050178000601410082
:109ef000430620000388b900000141008202780077
:109f00001e1f12001e971a001e00be00a200200095
:109f10000300200001e507000043b00092fd0700a8
:109f20001e00be00a200200003002000fbe407008a
:109f3000a20020000202b8000001eb000283b90079
:109f40000501780006014100a30020000388b90044
:109f500000014100820278001e1f12001e971a00a5
:109f60004e4090000004e00003003a0001c3b3003b
:109f70001ec040007cfd07000080fa0000000600c3
:109f80000400fa00008fbe0012c0b3001e00be0025
:109f900014ff07000080fa00000006000400fa0029
:109fa000008fbe00f0232400f1002000be0f10003f
:109fb000ae8f180003003400f0232400f1002000cd
:109fc000008fbe001e00be00026a280013002000a1
:109fd000d2e407000043b00063fd07001e00be008e
:109fe000026a280013002000cce40700026a28005f
:109ff0000202b800120020000283b90005017800b7
:10a0000006014100036a28000388b90000014100ed
:10a01000820278001e1f12001e971a001e00be004a
:10a020000271220003002000bce407000043b000de
:10a030004dfd07001e00be0002712200030020003b
:10a04000b6e40700027122000202b8000001eb0032
:10a050000283b90005017800060141000371220066
:10a060000388b90000014100820278001e1f12001f
:10a070001e971a001e00be00823e20000300200032
:10a08000a6e407000043b00037fd07001e00be0035
:10a09000823e200003002000a0e40700823e200052
:10a0a0000202b8000001eb000283b900050178004c
:10a0b00006014100833e20000388b90000014100f1
:10a0c000820278001e1f12001e971a00e0c2b30021
:10a0d00025fd07001e00be004206200003002000f0
:10a0e0008ee407000043b0001ffd07001e00be0005
:10a0f000420620000300200088e4070042062000fa
:10a100000202b8000001eb000283b90005017800eb
:10a1100006014100430620000388b9000001410008
:10a12000820278001e1f12001e971a001e00be0039
:10a13000a20020000300200078e407000043b000e4
:10a1400009fd07001e00be00a20020000300200041
:10a1500072e40700a20020000202b8000001eb0038
:10a160000283b9000501780006014100a300200028
:10a170000388b90000014100820278001e1f12000e
:10a180001e971a0001c3b3001ec04000f6fc070072
:10a190000080fa00000006000200fa00000f7800bc
:10a1a0001e00e00002003400b0c2b300eefc070065
:10a1b0001e00e00002003a0000c2b300eafc070003
:10a1c0001e00e00003003d00d0c2b300e6fc070023
:10a1d0001e0fea001e007800823e200011000900d8
:10a1e0000200d8000043b000dffc07001e0078002a
:10a1f000823e2000110009000200d8008000fd000e
:10a20000803e20000088b9001e0f1000e0c2b3009d
:10a21000d5fc07001e00780042062000110009004e
:10a220000200d8000043b000cffc07001e007800f9
:10a2300042062000110009000200d8008000fd0045
:10a24000400620000088b9001e0f10001e00780094
:10a25000a2002000110009000200d8000043b00055
:10a26000c1fc07001e007800a200200011000900b8
:10a270000200d8008000fd00a00020000088b90086
:10a280001e0f10000080fa00000006000600fa0011
:10a29000000f7800110798000000eb0020079800dd
:10a2a000f07022009e0f100002003400f0702200b7
:10a2b000000f78009e00900040072000808f500023
:10a2c000120032001e007800823e200011000900ba
:10a2d0000200d8000000e00005003a0000c2b30010
:10a2e000a1fc07001000200020079800090037009b
:10a2f0001e007800823e2000110009000200d800f4
:10a300000043b00098fc0700020037001000200056
:10a31000200798001e007800823e200011000900ee
:10a320000200d8008000fd00803e20000088b900b7
:10a330001e0f10002e009000e10f50000c003a009c
:10a340001e00780042062000110009000200d8001b
:10a350000000e00006003a001e009000e20f5000ee
:10a360000300320000c2b3007ffc07000600370084
:10a370001e00780042062000110009000200d800eb
:10a380000043b00078fc07001e0078004206200061
:10a39000110009000200d8008000fd0040062000e6
:10a3a0000088b9001e0f10001e009000e20f500040
:10a3b00002003a00e0c2b3006bfc07001e00780008
:10a3c000a2002000110009000200d8000043b000e4
:10a3d00065fc07001e007800a200200011000900a3
:10a3e0000200d8008000fd00a00020000088b90015
:10a3f0001e0f10001e009000e10f500002003a00f6
:10a40000e0c2b30058fc07009e00900070072000d7
:10a41000808f500003003a0070c5b30052fc070063
:10a420000300370001c3b3001ec040004efc07000c
:10a430000080fa00000006000200fa00004f7800d9
:10a4400090c0b3009e4f10000200340090c0b300d3
:10a45000004f780001c3b3001ec0400042fc07005b
:10a460000080fa00000006000200fa000000eb0085
:10a47000000f7800900020009e0f100006003c00a6
:10a48000c0c020009e00400000c2b3008048780099
:10a490001e0fe800f7ff37000040eb0015ecb70097
:10a4a0000080fa00000006000800fa00004f780063
:10a4b0001e80fb0030079800c00d2000be009000f9
:10a4c000808f500039003200c00d20003e01900006
:10a4d000800f510016003c00400c2000be00900090
:10a4e000808f500028003200400c20003e01900078
:10a4f000800f510005003c00c0052000be00900008
:10a50000808f50002c0032002e003700500c2000ad
:10a510003e019000800f510021003200600d2000ac
:10a52000be009000808f50001a00320025003700d6
:10a53000500e20003e019000800f510018003200a4
:10a54000500e2000be009000808f500005003c009f
:10a55000400e20003e019000800f51000a003200a2
:10a5600018003700600f2000be009000808f500060
:10a5700008003200c00f20003e019000800f510003
:10a580000a0032000f00370010ceb3004047980099
:10a590000e003700f0ceb300404798000b003700a4
:10a5a00010c6b300404798000800370050cfb300f2
:10a5b000404798000500370000c6b30040479800a8
:10a5c000020037001e407800404798000000eb0072
:10a5d000100798001e009000e60f50000b003c0092
:10a5e0001e009000c2c02000820040001e009000ab
:10a5f000d2c0200002004000904878001e00900069
:10a600000000e80010079800f2ff37004e4090006d
:10a6100013ecb7000080fa00000006000400fa0006
:10a62000060ce2004c00320043c62e002160800080
:10a63000800020000008b800126080000200400086
:10a6400003004000104f7800505c8000615c800087
:10a65000e00f5000e08f58003f003a001e00fb0062
:10a6600010079800d00220009e009000808f5000bc
:10a6700030003200d00220009e009000808f5000f9
:10a6800008003c001e0090000000e00009003200bd
:10a69000000220009e009000808f50000d003200cc
:10a6a00004003700e00220009e009000808f5000e0
:10a6b000250032000000eb0030608800005d800063
:10a6c0000000d000cf80de00505c8800615c880014
:10a6d00021003700106080000000e8001060880052
:10a6e000015d8000400020000088b900cf80de00be
:10a6f000505c8800615c8800005d8000cf80de00d7
:10a70000c25c80000012b800c25c80000193b900f6
:10a710000501780006014100d35c80000380b90088
:10a720000001410082027800e45c8800f55c88004a
:10a7300009003700106080000000e8001060880009
:10a740009ff6070004003700106080000000e8005a
:10a750001060880064f607000080fa000000060020
:10a760000600fa00004f78001e80fb0020079800ca
:10a77000c00d2000ae009000808f500035003200e8
:10a78000c00d2000ae009000808f500012003c00f1
:10a79000500c2000ae009000808f50002a00320044
:10a7a000500c2000ae009000808f500005003c004f
:10a7b000400c2000ae009000808f50001c00320042
:10a7c00027003700600d2000ae009000808f500001
:10a7d0001a00320022003700500e2000ae00900018
:10a7e000808f500018003200500e2000ae00900004
:10a7f000808f500005003c00400e2000ae0090000d
:10a80000808f50000a00320015003700600f2000d2
:10a81000ae009000808f500008003200c00f200072
:10a82000ae009000808f50000a0032000c0037000c
:10a8300000042000100798001700370010042000c3
:10a84000100798001400370020042000100798001b
:10a850001100370030042000100798000e00370068
:10a86000f0c1b3009e4f100002003e0000c2b300d2
:10a87000004f7800f0c5b3009e4f10000200360074
:10a8800000ceb3001e4f40001e80fb0001fe2f00d3
:10a8900001004000100798001e0090000080fa00a0
:10a8a000000006000200fa00004f7800060ce200eb
:10a8b000feff3a001e407800a9ff070020608800d4
:10a8c0000000eb001060880010002000306088005d
:10a8d0000080fa00000006000200fa00000f780075
:10a8e0000000eb00a04288001e0078001004e00089
:10a8f0000f0032001e007800d1c0b30090cf1000ce
:10a900000b0032001e00780010407800e6fe0700c1
:10a910001e00780010407800e2ff07001e0078005b
:10a920001000fb0040f907001e0fe800eeff3700a3
:10a930000080fa00000006000200fa00000f780014
:10a940001e007800b06088001e007800c06088009b
:10a950000000eb00d0608800c3fe07000080fa0012
:10a96000000006000600fa00060ce20029013a0089
:10a97000c0608000104f78001e04e0000300320029
:10a98000d0c0b3009e4f100012003a00b1608000aa
:10a99000c16088007609e20019013400b04b8000e4
:10a9a0000000e900b04b88007609e20014013a008b
:10a9b000a000200001002000e05c8800f15c88001d
:10a9c000d04c8000cf80de00c05c8800d15c880065
:10a9d0000b013700c06080000000e800c060880004
:10a9e000d260800022079800ae019000e28f5100f3
:10a9f0006c0032002e009000e20f500007003c0077
:10aa0000ae0090000100e0000d0032002e01900029
:10aa1000e10f51001800320009003700ae0190002c
:10aa2000e48f51009b0032002e009000e30f500095
:10aa300062003400ae009000e58f5000e10032006b
:10aa4000c0c5b3009e4f100003003a001000200064
:10aa5000d0608800e80037001e40780040ff070003
:10aa6000206088000000eb001060880010002000cb
:10aa700030608800e00037001e01fb0012079800dc
:10aa8000800520009e019000808f51003f00320021
:10aa9000800520009e009000808f500012003c0036
:10aaa000000520001e019000800f5100240032009c
:10aab000000520009e019000808f510005003c00a1
:10aac000600420009e009000808f5000270032001c
:10aad00031003700300520001e019000800f51002a
:10aae0001a0032002c003700000720009e01900061
:10aaf000808f510012003200000720009e0090005d
:10ab0000808f500005003c00600620001e01900070
:10ab1000800f5100150032001f0037003007200061
:10ab20009e019000808f51000800320080072000b5
:10ab30009e009000808f50001400320016003700f5
:10ab400020002000d0608800ab00370030002000db
:10ab5000d060880030002000e06088006000b8000d
:10ab60004060880051608800a3003700400020004a
:10ab7000d060880060002000e06088006000b800bd
:10ab800040608800516088009b0037005000200022
:10ab9000d0608800980037000000eb00d06088008b
:10aba000950037001e00fb0063006000b04a88007b
:10abb0000000eb00d06088008f0037001c0ce20022
:10abc0008d0034004060800051608000a2002000b1
:10abd0000203b8000001eb000282b900070178000f
:10abe00004014100a30020000388b90000014100d6
:10abf000820378001e4078000000fb00cf80de005a
:10ac00006f0060008000eb0006034000878348006f
:10ac10004660880057608800e06080000000e9001e
:10ac2000e06088001c0ce20073003a004060800085
:10ac300051608000e00f5000e08f580004003c009d
:10ac40001000200001002000406088005160880052
:10ac50004260800053608000401f200001002000ff
:10ac6000800f5100818f590004003400401f2000e4
:10ac70000100200040608800516088004260800030
:10ac8000e24a8800cde907000000eb00d0608800b0
:10ac9000590037001c0ce20057003400406080006f
:10aca00051608000a20020000203b8000001eb0008
:10acb0000282b9000701780004014100a3002000ce
:10acc0000388b90000014100820378001e4078002b
:10acd0000000fb00cf80de006f0060008000eb0012
:10ace000060340008783480046608800576088005c
:10acf000e06080000000e900e06088001c0ce200d9
:10ad00003d003a0062de2d005142800040002000ec
:10ad10000008b800000141004060800051608000e0
:10ad2000b20f5000a28f58000800340062de2d00e0
:10ad300051428000400020000008b800000041009f
:10ad40001001be004260880053608800a2dd2d0023
:10ad500051428000400020000008b800000141007e
:10ad60004060800051608000b20f5000a28f5800f8
:10ad700008003d00a2dd2d0051428000400020006f
:10ad80000008b800000041001001be0042608800c9
:10ad90005360880051428000400020000008b80045
:10ada000a3942000030040004260800053608000b4
:10adb0000288be00f1e507000000eb00d0608800cb
:10adc0000d0037001e00fb00610060000000e00085
:10add00004003200c4e2a80010002000c04b88002c
:10ade00003003700c4e2a9000000eb00c04b88005c
:10adf0000000eb00d06088001e407800aafd07002c
:10ae0000304b8000e10f500002003a001e00fb00b2
:10ae100005f807000080fa00000006000600fa00ae
:10ae200020002000200798006000b800008fbe00be
:10ae3000ae00900080618000808f500019003d00be
:10ae40001e00be00a20020000203b8000001eb00bb
:10ae50000282b9000701780004014100a30020002c
:10ae60000388b90000014100820378002e009000a1
:10ae700021c3200001004000104078000000fb00ca
:10ae8000cf80de006f0060008000eb00001f4300f9
:10ae900001974b002e0090000000e800200798006a
:10aea000e3ff37001e00be000080fa00000006002d
:10aeb0000000fa007209f80040e82e00801f7800b8
:10aec0003ed50700e48757000080fa000000060026
:10aed0000000fa0051428000400020000008b80045
:10aee000a2942000020040001001be00829fbe001c
:10aef000b0e82e00801f780030d50700e6875700a5
:10af00000080fa00000006000000fa0060428000a5
:10af1000e10f500005003a0050e92e00801f780034
:10af200026d507008f87e90004003700b0e92e001e
:10af3000801f780021d507008f87e9000080fa0084
:10af4000000006000000fa006009f80010ea2e0078
:10af5000801f780019d50700e48757000080fa00a9
:10af6000000006000000fa005c09f80080ea2e00ec
:10af7000801f780011d50700e48757000080fa0091
:10af8000000006000000fa005609f80010eb2e0041
:10af9000801f780009d50700e48757000080fa0079
:10afa000000006000000fa007809f80080eb2e008f
:10afb000801f780001d50700e48757000080fa0061
:10afc000000006000000fa005809f800f0eb2e001f
:10afd000801f7800f9d40700e48757000080fa004a
:10afe000000006000000fa005a09f80060ec2e008c
:10aff000801f7800f1d40700e48757000080fa0032
:10b00000000006000200fa0080852000000f780092
:10b01000d0ec2e00801f7800e8d407008f87e9006d
:10b020001e0078001004e000090032001e007800c5
:10b03000d1c0b30090cf1000050032001e00780090
:10b040001040780078f707001e0fe800f4ff370083
:10b0500000ed2e00801f7800d8d407008f87e9000c
:10b060000080fa00000006000a00fa0034ccbf009d
:10b070000000fb004007980090042000ce009000e4
:10b08000808f500015003200900420004e01900087
:10b09000800f510009003c0020042000ce009000e9
:10b0a000808f50005d003200400420004e0190006f
:10b0b000800f5100760032000800370000052000a4
:10b0c000ce009000808f5000370032003005200005
:10b0d0004e019000800f51004a00320030ed2e00ea
:10b0e000801f7800b5d407008f87e90050428000a8
:10b0f00030079800be009000e18f5000070032003a
:10b100003e019000e10f51000e0034003e0090001f
:10b11000e20f5000060032000a00370070ed2e00ea
:10b12000801f7800a5d407008f87e9000900370049
:10b1300020ee2e00801f7800a0d407008f87e90042
:10b1400004003700d0ee2e00801f78009bd407004b
:10b150008f87e90050ef2e00801f780097d40700fa
:10b160008f87e90080d82d00801f780093d40700d6
:10b170008f87e900b0ef2e00801f78008fd4070082
:10b180008f87e900e0d82d00801f78008bd407005e
:10b190008f87e90000ed2e00801f780087d407001c
:10b1a0008f87e90050003700e1418000a04c80000b
:10b1b000000ab800e1418000b04c80000088b9006e
:10b1c0000501780000014100a14c8000f0418000a1
:10b1d0000088b900000141008202780040a8de002a
:10b1e000cf80de00000f78009e007800811f78007d
:10b1f00030f02e00801f780070d40700e4875700dd
:10b20000390037004408f800b0f02e00801f7800a5
:10b210006ad40700e487570033003700a0002000fd
:10b22000b6e40700cf80de00624c80000012b80058
:10b23000624c80000193b9000501780006014100cd
:10b24000734c80000380b900000141008202780045
:10b2500014079800250798001e009000ae0090008b
:10b260004809dd004800de0000007100c888de00eb
:10b27000000f78001e007800801f780030f12e004b
:10b28000801f78004dd40700e48757001600370070
:10b290009000200099e40700cf80de00424c80003f
:10b2a0000202b800524c80000283b9000501780008
:10b2b00006014100434c80000198b90000014100a3
:10b2c0008202780040a8de00cf80de00000f780008
:10b2d0009e007800811f7800b0f12e00801f78005a
:10b2e00036d40700e48757000080fa00000006000b
:10b2f0000000fa00b04b8000e10f400005003a006a
:10b3000030f22e00801f78002cd407008f87e900d0
:10b31000050037007609f80090f22e00801f7800b3
:10b3200026d40700e48757000080fa0000000600da
:10b330000400fa00b9fe0700008fbe00a2dd2d0058
:10b3400051428000400020000008b8000000410089
:10b350001e01be00b00f5100a08f59000700310040
:10b36000a2dd2d0051428000400020000008b800fe
:10b37000000041001001be00028fbe0062de2d0001
:10b3800051428000400020000008b8000000410049
:10b390001e01be00b00f5100a08f590007003600fb
:10b3a00062de2d0051428000400020000008b800fd
:10b3b000000041001001be00028fbe00514280001b
:10b3c000400020000008b800a394200003004000c3
:10b3d0001e01be000288be0068e407000080fa007b
:10b3e000000006000200fa008cfe0700000f780043
:10b3f0001e00e00002003d000000eb00000f78009e
:10b40000200020009e0f10000200340020002000c9
:10b41000000f78001e007800904b88000080fa0032
:10b42000000006000200fa007cfe0700000f780012
:10b430001e00e00002003d000000eb00000f78005d
:10b44000400020009e0f1000020034004000200049
:10b45000000f78001e007800004b8800004b800031
:10b46000e40f5000020032000000eb00b04b8800f7
:10b470000080fa00000006000200fa0067fe0700e4
:10b48000000f78001e00e00002003c0010002000c9
:10b49000000f7800401f20009e0f100002003400b3
:10b4a000401f2000000f78001e007800e04a88004e
:10b4b000c2e707000080fa00000006000200fa0060
:10b4c00056fe0700000f78001e00e00002003d005d
:10b4d0000000eb00000f7800300020009e0f1000ed
:10b4e0000200340030002000000f78001e007800b9
:10b4f000b04a88000080fa00000006000200fa004e
:10b5000046fe0700000f78001e00e00002003d002c
:10b510000000eb00000f7800100020009e0f1000cc
:10b520000200340010002000000f78001e00780098
:10b53000c04b88000080fa00000006000200fa00fc
:10b5400036fe0700000f78001e00e00002003d00fc
:10b550000000eb00000f7800200020009e0f10007c
:10b560000200340020002000000f78001e00780048
:10b57000c04a88000080fa00000006000200fa00bd
:10b5800026fe0700000f78001e00e00002003d00cc
:10b590000000eb00000f7800100020009e0f10004c
:10b5a0000200340010002000000f78001e00780018
:10b5b000d04a88000080fa00000006000200fa006d
:10b5c0000080fa00000006000200fa00004f780038
:10b5d000e062800081852000010040001e48780064
:10b5e000e1628000c00e2000808f500003003c000c
:10b5f000e06280000000e800e06288000080fa005d
:10b60000000006000000fa00e06280008285200051
:10b6100082004000d0c0b30080487800e062800023
:10b620000000e800e0628800e0628000828520007f
:10b63000820040000040eb008048780080852000b8
:10b64000bdfc07000000eb00d06288000080fa001b
:10b65000000006000200fa0000c3b300344ce3000f
:10b6600011003a000000eb00b04b88000000eb0036
:10b67000306088000000eb00405c88000400fc00a3
:10b680006000b800505c8800615c880081f20700af
:10b690000400fc006000b800e05c8800f15c8800f9
:10b6a00025f207002e0037007609e2002c003a0050
:10b6b000904b8000b0628800014b8000a16288003e
:10b6c0000000eb00c062880010002000904b880052
:10b6d00040002000004b88008085200096fc070079
:10b6e00034ccbf000000fb00000f780010032000e6
:10b6f0009e007800808f50001900350090032000d4
:10b700009e007800808f500011003400300420002b
:10b710009e007800808f5000050032004005200018
:10b720009e007800808f5000040032000c0037002b
:10b730000080eb00b04b88000900370010002000ab
:10b74000c062880010002000b04b88000400370061
:10b7500034ccbf000000fb006f006000b04b8800dd
:10b760000080fa00000006000200fa000000eb0072
:10b77000000f7800700020009e0f100006003c00b3
:10b7800020c320009e0040000040eb00804878006d
:10b790001e0fe800f7ff37000000eb008061880013
:10b7a0000000eb00d06288000000eb00e06288003f
:10b7b0000080fa00000006000400fa00004f780044
:10b7c0001e04e00003003200a0c0b3009e4f100032
:10b7d00003003a0010002000100798000200370014
:10b7e0000000eb00100798001e0090000080fa0097
:10b7f000000006000e00fa000000000099f50700a6
:10b800000000e000c0003200a6f50700004f7800fd
:10b810001e407800e8ff07000000e000ba003a0090
:10b82000d0c3b3009e4f100003003200f0c3b3003a
:10b830009e4f100006003a005a0ce20004003a0045
:10b8400080618000e20f500001003400c6ff070055
:10b85000d0c0b3009e4f100095003a0032ccbf001c
:10b860000000fb0060079800d0032000ee0090006d
:10b87000808f500048003200f00320006e019000dd
:10b88000800f510088003a0033ccbf000001fb005c
:10b89000cf91de00f0fb2f00f1ff2f0002014000ee
:10b8a0008381480022079800330798007001200028
:10b8b000010020002e019000be019000800f510079
:10b8c000818f590032003e002e009000be00900093
:10b8d00000600100250037002a00370025003700ee
:10b8e0002b0037002a0037001200370028003700ed
:10b8f00027003700250037002500370013003700e8
:10b90000230037001d003700210037000b003700ef
:10b91000120037001e0037001d0037000d003700f1
:10b92000080037001a0037001900370018003700e8
:10b930000c00370066fd0700150037005cfd0700ae
:10b940001300370070fd0700110037007dfd070070
:10b950000f00370083fd07000d00370089fd070049
:10b960000b0037008ffd07000900370095fd070029
:10b97000070037009bfd070005003700a1fd070009
:10b98000030037005afe070001003700b6fd07002c
:10b9900075ff070099ff370033ccbf000001fb00a3
:10b9a000cf91de00f0fb2f00f1ff2f0002014000dd
:10b9b00083814800420798005307980070012000d7
:10b9c000010020004e019000de019000800f510028
:10b9d000818f590032003e004e009000de00900042
:10b9e00000600100250037002a00370025003700dd
:10b9f0002b003700290037001400370028003700db
:10ba000027003700260037002500370013003700d5
:10ba1000230037001d0037002100370009003700e0
:10ba2000120037001e0037001d0037000d003700e0
:10ba3000080037001a0037001900370018003700d7
:10ba40000c00370067fe07001500370038fe0700be
:10ba500013003700d9fe07001100370071fe070000
:10ba60000f00370084fe07000d00370093fe07002b
:10ba70000b003700a1fe070009003700affe0700ea
:10ba800007003700bdfe070005003700ddfe070098
:10ba900003003700effe070001003700c5e3070091
:10baa00031ff070055ff37002fff070053ff370016
:10bab000d0c3b300324ce30008003a00d0c4b30056
:10bac000334ce30005003a0010002000d0628800eb
:10bad0001e407800bcfe070048ff370080618000f0
:10bae00021c32000010040001e48780080618000d2
:10baf000ee0f500041ff3c00806180000000e80034
:10bb0000806188003dff37000080fa0000000600d9
:020000040000fa
:0200000401f009
:04000000e5ff000018
:020000040000fa
:0200000401f009
:04000400ff7f00007a
:020000040000fa
:0200000401f009
:04000800ffff0000f6
:020000040000fa
:0200000401f009
:04000c00ffff0000f2
:020000040000fa
:0200000401f009
:04001000ffff0000ee
:020000040000fa
:0200000401f009
:04001400ffff0000ea
:020000040000fa
:1000080064460000184500004e45000026460000e2
:100018004c46000064460000644600006446000048
:100028006446000064460000644600006446000020
:100038006446000064460000644600005a4100001f
:1000480064460000964600006446000064460000ce
:1000580064460000644600006446000064460000f0
:1000680064460000644600006446000064460000e0
:1000780064460000644600006446000064460000d0
:1000880064460000644600006446000064460000c0
:1000980064460000644600006446000064460000b0
:1000a80064460000644600006446000064460000a0
:1000b8006446000064460000644600006446000090
:1000c8006446000064460000644600006446000080
:1000d8006446000064460000644600006446000070
:1000e8006446000064460000644600006446000060
:0800f8006446000064460000ac
:020000040000fa
:1001080064460000184500004e45000026460000e1
:100118004c46000064460000644600006446000047
:10012800644600006446000064460000644600001f
:100138006446000064460000644600005a4100001e
:1001480064460000964600006446000064460000cd
:1001580064460000644600006446000064460000ef
:1001680064460000644600006446000064460000df
:1001780064460000644600006446000064460000cf
:1001880064460000644600006446000064460000bf
:1001980064460000644600006446000064460000af
:1001a800644600006446000064460000644600009f
:1001b800644600006446000064460000644600008f
:1001c800644600006446000064460000644600007f
:1001d800644600006446000064460000644600006f
:1001e800644600006446000064460000644600005f
:0801f8006446000064460000ab
:020000040000fa
:10bb1000763100002e300000330000003137000085
:10bb20002e310000302e000032300000303900008d
:10bb30000031000032300000302000002000000002
:10bb400000320000343000003020000020000000ef
:10bb500000340000383000003020000020000000d9
:10bb600000390000363000003020000020000000c6
:10bb700000310000393200003030000020000000a9
:10bb80000033000038340000303000002000000096
:10bb90000035000037360000303000002000000083
:10bba000003100003135000032300000302000004c
:10bbb00000000000c0d4000001000000a0680000e8
:10bbc00006000000c0d4000001000000c0270000f3
:10bbd00009000000c02700000900000030e6000056
:10bbe000020000000a0d0000576f000072640000a0
:10bbf000732000003d200000256400002c20000080
:10bc0000537500006365000073730000203d000061
:10bc100020250000642c000020430000686500001f
:10bc2000636b0000737500006d2000003d20000074
:10bc300025580000000a00000d5700006f72000038
:10bc400064730000203d000020250000642c0000eb
:10bc500020530000756300006365000073730000eb
:10bc6000203d000020250000642c0000204300003f
:10bc700068650000636b0000737500006d200000b4
:10bc80003d20000025580000007600007676000078
:10bc90002076000076760000206400006520000019
:10bca0004a5500004d41000020420000656100003f
:10bcb000636f00006e200000232000000d000000d4
:10bcc00050570000522000004d4900004e00000077
:10bcd00050570000522000004c4f00005700000059
:10bce000505700005220000020480000490000008a
:10bcf00050570000522000004d4100005800000045
:10bd000050570000522000003f3f00003f0000005d
:10bd10002020000020200000200000002053000010
:10bd20005752000020000000204300005552000040
:10bd300052000000203f00003f3f00003f00000095
:10bd40005057000052000000490000004100000070
:10bd5000492000002d2d00002e2d00004100000084
:10bd600050770000722000004f460000462000007f
:10bd70006166000074650000722000002569000003
:10bd800020200000002000002020000020200000d3
:10bd900020200000202000002020000020200000a3
:10bda00020200000200000000a0d00005573000054
:10bdb0006572000020730000657400007469000063
:10bdc0006e6700007320000073610000766500005c
:10bdd00064200000746f0000204500004550000002
:10bde000524f00004d2c0000205000006f770000e3
:10bdf00065720000206f0000666600000a0d0000fa
:10be000000430000572e0000252e00003164000082
:10be100000430000572500002e320000640000009f
:10be200052530000323300003220000054650000fd
:10be3000737400002020000020200000202000005b
:10be40000057000061690000746900006e6700001f
:10be50002064000061740000612e00002e2e00009e
:10be60002e000000525800002064000061740000a1
:10be70006120000020000000202000003078000039
:10be8000004a0000554d00004120000054580000b9
:10be90003530000030200000004a0000554d000001
:10bea00041200000545800003133000036200000cb
:10beb000004a0000554d0000412000003f3f0000b7
:10bec0003f3f00003f20000000200000204f000006
:10bed000483200004e4c0000542000004f48000043
:10bee000375300005620000020000000536500007a
:10bef0007276000069630000652000004d6f00004d
:10bf00006465000020200000202000000050000098
:10bf10007573000068200000444900005350000081
:10bf20004c410000592000006e78000074000000b1
:10bf30005075000073680000204f0000504500005d
:10bf4000522000003d200000536100007665000093
:10bf5000000a00000d45000045500000524f00004f
:10bf60004d20000063680000656300006b730000f3
:10bf7000756d0000732c000020430000616c000010
:10bf8000203d000020250000582c00002044000027
:10bf90006566000020430000732000003d20000083
:10bfa000255800002c20000046610000637400004a
:10bfb0006f72000079200000646500006661000077
:10bfc000756c00007420000072650000736500004d
:10bfd00074730000203d0000202500006400000074
:10bfe0000a0d000045450000505200004f4d000072
:10bff0002063000068650000636b0000737500003b
:10c000006d20000065720000726f0000722c00004d
:10c0100020720000656c00006f6100006420000069
:10c0200066610000637400006f72000079200000f8
:10c030006465000066610000756c000074730000a8
:10c040000050000075730000682000005345000098
:10c0500054200000666f00007220000020200000c5
:10c060002000000066610000637400006f72000031
:10c07000792000006465000066610000756c0000b6
:10c0800074730000000a00000d0a00000d4a000051
:10c09000554d00004120000054580000353000008c
:10c0a000302000002f200000000a00000d0a0000d0
:10c0b0000d4a0000554d000041200000545800007a
:10c0c00031330000362000002f200000000a00005d
:10c0d0000d0a00000d4a0000554d000041200000ef
:10c0e000556e00006b6e00006f7700006e20000040
:10c0f0004d610000696e0000204200006f61000089
:10c10000726400002074000079700000652f000048
:10c1100020000000202f0000200000000a0d000079
:10c12000436f0000707900007269000067680000ca
:10c13000742000004a75000068610000204e000075
:10c14000696900006e6900006b6f0000736b00008e
:10c15000692c0000204f0000483200004e4c0000c7
:10c16000540a00000d0a00000d0000005379000081
:10c1700073740000656d0000204300006c6f0000c8
:10c18000636b0000203d00002025000069200000b6
:10c190006b4800007a0a00000d0000000a0d000044
:10c1a0005365000074200000554100005254000007
:10c1b00020750000736500007220000062610000bd
:10c1c00075640000207200006174000065200000aa
:10c1d000746f000020230000256900002c2000005f
:10c1e0002025000073620000640a00000d000000ba
:10c1f0000a0d000043570000206200007265000035
:10c20000616b000020740000696d00006520000073
:10c210007365000074200000746f0000202500008a
:10c2200069200000756e0000697400007300000052
:10c230000a0d00000a0d0000556e00006b6e000034
:10c240006f7700006e2000006d610000696e0000d5
:10c25000206200006f610000726400002074000022
:10c2600079700000652c00002070000072650000ed
:10c2700073730000204f0000504500005220000062
:10c28000746f0000206300006f6e0000746900008e
:10c290006e75000065200000616e00007977000077
:10c2a000617900000a0d0000004f000050450000b9
:10c2b000522000003d200000436f00006e7400001b
:10c2c000696e00007565000020000000204200003b
:10c2d00045410000434f00004e20000020000000b8
:10c2e0005357000052000000204e00002f41000074
:10c2f0002000000020000000560000002020000068
:10c30000545800002020000000200000535400007a
:10c310004259000020000000204f0000504500005e
:10c320005220000000200000545500004e4500003f
:10c33000200000005072000065200000416d0000e8
:10c34000706c0000696600006965000072200000e2
:10c350002020000000530000656c000065630000b1
:10c36000742000003d200000004f00004646000001
:10c370002020000020200000003100003064000078
:10c380004220000020200000003200003064000045
:10c390004220000020200000003f00003f3f00003e
:10c3a0004d4800007a200000636f00006e760000a8
:10c3b000657200007465000072000000332e0000fa
:10c3c000354d0000487a0000206300006f6e0000c9
:10c3d0007665000072740000657200000031000094
:10c3e000304d0000487a0000206300006f6e0000ae
:10c3f000766500007274000065720000004f000056
:10c400004e200000202000002020000000430000fb
:10c41000572000005369000064650000746f00003d
:10c420006e65000020200000202000002000000099
:10c43000546f00006e650000203d0000204f00009a
:10c4400046460000202000002020000020200000a0
:10c45000005400006f6e0000652000003d200000c9
:10c4600025690000487a00002020000020200000fc
:10c470002020000000530000575200002050000010
:10c48000726f000074200000004c0000696d000015
:10c4900069740000203d0000200000002020000002
:10c4a00020200000004b000065790000657200004c
:10c4b000207400007970000065200000202000003a
:10c4c00020200000200000004b650000796500007e
:10c4d000722000003d200000446f00007420000026
:10c4e00070720000692e0000004b000065790000aa
:10c4f00065720000203d000020490000616d0000d1
:10c500006269000063200000410000004b650000ec
:10c5100079650000722000003d20000049610000a4
:10c520006d6200006963000020420000004b0000c3
:10c530006579000065720000203d00002053000076
:10c5400074720000616900006768000074000000f8
:10c550004b65000079650000722000003d2000005e
:10c5600042650000616300006f6e00002020000043
:10c570000044000069730000706c0000204200005d
:10c580007269000067680000746e00006573000047
:10c59000730000004c43000044200000424c0000a7
:10c5a000203d000020250000692000002020000020
:10c5b000202000002000000044690000737000008b
:10c5c0006c61000079200000436f00006e74000071
:10c5d0007261000073740000004300006f6e000081
:10c5e0007472000061730000742000003d200000a0
:10c5f0002569000020200000005300006572000043
:10c60000696100006c200000507200006f7400002f
:10c610006f6300006f6c00002000000052530000a8
:10c6200032330000322000003d000000545800006a
:10c6300031330000362f000035300000300000009c
:10c6400020540000657200006d6900006e610000fa
:10c650006c0000005365000072690000616c00000e
:10c660002053000070650000656400002020000079
:10c6700020200000004200006175000064200000de
:10c6800052610000746500003d2500007300000049
:10c6900054580000204300006f6e000074720000c8
:10c6a0006f6c0000202000002020000020200000ef
:10c6b00000410000757400006f2000002020000081
:10c6c000004d00004f5800002020000020200000f6
:10c6d0000053000050410000524500002049000076
:10c6e0002f4f000020730000696700006e6100009a
:10c6f0006c000000447500006d70000020450000d3
:10c7000045500000524f00004d200000636f0000b4
:10c710006e740000656e0000747300000a0d000066
:10c72000000a00000d250000352e000034580000de
:10c730000020000025340000580000000a0d000011
:10c740004c610000737400002073000075630000ea
:10c750006365000073730000206300006f640000d5
:10c76000652000003d20000025580000200000004a
:10c770000a0d00004d6f000072730000652000007c
:10c78000436f000064650000207000006c610000d1
:10c790007965000072200000746500007374000069
:10c7a0002c2000006d6f000064650000203d00003b
:10c7b00020250000640a00000d0000000a0d0000a2
:10c7c0005772000069740000652000006d6500006c
:10c7d0007373000061670000652000006d61000058
:10c7e00078200000266400002063000068610000db
:10c7f000722c000020740000657200006d6900005a
:10c800006e6100007465000020770000697400000c
:10c8100068200000435200000a0d0000000a0000da
:10c820000d5000006c61000079200000737400005e
:10c830006172000074650000640a00000d000000d1
:10c840000a0d0000577200006974000065200000a6
:10c8500042650000616300006f6e0000206d000003
:10c86000657300007361000067650000206d0000c3
:10c87000617800002025000064200000636800004b
:10c88000617200002c20000074650000726d0000d1
:10c89000696e000061740000652000007769000087
:10c8a0007468000020430000520a00000d000000e0
:10c8b0000a0d0000000a00000d2d00002d2d0000c3
:10c8c0002042000065610000636f00006e200000e0
:10c8d000636f00006e740000726f00006c20000037
:10c8e000636f00006d6d0000616e000064730000f6
:10c8f000202d00002d2d00000a0d00000062000018
:10c90000205700007269000074650000204200009a
:10c9100065610000636f00006e2000006d6500001f
:10c920007373000061670000650a00000d000000dd
:10c930007020000050720000696e0000742000003a
:10c9400042650000616300006f6e0000206d000012
:10c950006573000073610000676500002c20000013
:10c960006e6f0000207300006f7500006e640000a1
:10c970000a0d0000007400002054000065730000e0
:10c9800074200000706c00006179000020420000fb
:10c9900065610000636f00006e2000006d6500009f
:10c9a0007373000061670000650a00000d0000005d
:10c9b00073200000537400006172000074200000b6
:10c9c00042650000616300006f6e0000207400008b
:10c9d000726100006e7300006d69000073730000e7
:10c9e000696f00006e0a00000d0000007120000059
:10c9f000537400006f700000204200006561000069
:10ca0000636f00006e20000074720000616e000011
:10ca1000736d000069730000736900006f6e0000a1
:10ca20000a0d0000000a00000d2d00002d2d000051
:10ca3000205400006573000074200000636f000044
:10ca40006d6d0000616e000064730000202d000019
:10ca50002d2d00000a0d0000006900002073000069
:10ca600079730000746500006d200000696e00009d
:10ca7000666f00000a0d00000065000020640000e1
:10ca8000756d000070200000454500005052000008
:10ca90004f4d00000a0d00000063000020630000fd
:10caa0006c650000617200002045000045500000e8
:10cab000524f00004d2000006661000063740000ca
:10cac0006f7200007920000072650000736500003d
:10cad00074200000636f0000756e00007465000034
:10cae000720a00000d000000612000007368000061
:10caf0006f770000206100006c6c00002041000096
:10cb00004443000020760000616c00007565000061
:10cb1000730a00000d00000064200000444400007f
:10cb200053200000636f00006e730000746100000a
:10cb30006e740000730a00000d0000005420000015
:10cb4000706c000061790000207400006f6e0000be
:10cb5000650a00000d0000005720000077720000f9
:10cb600069740000652000004c4300004420000070
:10cb700074650000737400002048000045580000f0
:10cb80000a0d0000007700002077000072690000a5
:10cb900074650000204c0000434400002074000035
:10cba00065730000742000004153000043490000f9
:10cbb000490a00000d000000422000004c43000024
:10cbc00044200000626100007220000067720000d3
:10cbd000617000006820000074650000737400003c
:10cbe0000a0d0000005a00002043000050550000cc
:10cbf00020650000727200006f7200002074000057
:10cc00007261000070200000746500007374000001
:10cc10000a0d0000000a00000d0a00000d4200008d
:10cc200065610000636f00006e20000073740000f7
:10cc3000726900006e67000020660000726f0000dd
:10cc40006d2000007468000065200000454500006c
:10cc5000505200004f4d00003a0000000a0d000045
:10cc60000a0d0000257300000a0d0000000a0000f4
:10cc70000d5400006573000074200000506c00002b
:10cc8000617900002042000065610000636f0000d0
:10cc90006e20000073740000726900006e6700006f
:10cca0003a0a00000d0000000a0d00004265000075
:10ccb000616300006f6e00002054000058200000e7
:10ccc000737400006172000074650000640a000063
:10ccd0000d0000000a0d00004265000061630000c5
:10cce0006f6e000020540000582000007374000094
:10ccf0006f70000070650000640a00000d00000005
:10cd00000a0d00000a0d00004a5500004d410000c8
:10cd10002d54000058350000303000002063000022
:10cd20006f7000007972000069670000687400008d
:10cd3000204f000048370000535600002026000016
:10cd4000204f0000483200004e4c0000540a000002
:10cd50000d0000000a0d00000a0d00004a550000f9
:10cd60004d4100002d5400005831000033360000c2
:10cd7000206300006f700000797200006967000096
:10cd800068740000204f0000483700005356000030
:10cd900020260000204f0000483200004e4c0000ca
:10cda000540a00000d0000000a0d00000a0d0000ea
:10cdb000556e00006b6e00006f7700006e20000063
:10cdc0004d610000696e0000204200006f610000ac
:10cdd000726400002074000079700000652000007b
:10cde000636f0000707900007269000067680000de
:10cdf000742000004f480000375300005620000008
:10ce0000262000004f480000324e00004c54000025
:10ce10000a0d0000000a00000d5300006f660000bc
:10ce200074770000617200006520000076650000e4
:10ce300072730000696f00006e2000000020000087
:10ce40002f200000002c0000206300006f70000005
:10ce5000797200006967000068740000204a0000d1
:10ce600075680000612000004e690000696e0000d6
:10ce7000696b00006f7300006b690000204f0000b9
:10ce8000483200004e4c0000540a00000d00000023
:10ce90000a0d000041440000432000002569000005
:10cea000203d0000202500006900000045450000ed
:10ceb000505200004f4d00002072000065730000ca
:10cec00065740000206300006f7500006e74000040
:10ced00065720000206300006c6500006172000054
:10cee000656400000a0d0000004c0000434400008f
:10cef0002077000072690000746500002061000066
:10cf000073630000696900002c2000004553000095
:10cf1000432000003d200000656e000064200000fa
:10cf200074650000737400002c2000004352000060
:10cf3000203d0000206300006c650000617200006d
:10cf4000204c000043440000200a00000d000000b7
:10cf50006368000061720000203d00002025000091
:10cf6000780a00000d0000004c430000442000003f
:10cf70007772000069740000652000006865000099
:10cf8000782c0000203000007831000042200000a2
:10cf90003d200000656e0000642000007465000004
:10cfa000737400002c200000307800003044000032
:10cfb000203d0000206300006c65000061720000ed
:10cfc000204c0000434400000a0d00000020000037
:10cfd0003d200000256300000a0d000000620000f3
:10cfe000617200002067000072610000706800003c
:10cff0002074000065730000740a00000d0000003a
:10d000000a0d0000446900007620000062790000eb
:10d01000205a0000657200006f0000000a0d000039
:10d02000536f0000756e00006420000074650000fe
:10d03000737400002c20000046430000594d00008e
:10d04000487a0000202f0000207400006f6e00005e
:10d0500065280000487a0000292000002a200000ee
:10d06000322c000020670000697600006520000077
:10d07000706900007463000068200000000a00006e
:10d080000d5300006f7500006e64000020740000f6
:10d0900065730000742c00002067000069760000b2
:10d0a0006520000064750000726100007469000072
:10d0b0006f6e0000286d0000732900002000000042
:10d0c0000a0d000052650000662000006f7300002a
:10d0d00063200000256c0000642c00002068000024
:10d0e0007a5f00006269000074200000256600007d
:10d0f000000a00000d540000657300007420000059
:10d1000062650000616300006f6e00002070000027
:10d11000726900006d6900007469000076650000a6
:10d12000732c000020670000697600006520000075
:10d130006c6500007474000065720000206f0000d0
:10d14000722000006e7500006d62000065720000c4
:10d15000200000002c20000030780000252e000068
:10d16000325800000a0d0000000a00000d530000b4
:10d17000657400002052000065660000206f00000a
:10d180007363000020660000726500007175000086
:10d19000656e000063790000203e00002000000062
:10d1a0000a0d000054650000737400002c2000007c
:10d1b0006b65000079650000722000007469000052
:10d1c0006d6900006e670000200000000a0d00007d
:10d1d00062750000737900005f6300006f750000e6
:10d1e0006e74000065720000202000002025000001
:10d1f0006c640000000a00000d630000775f00000f
:10d2000062720000656100006b5f000074690000dd
:10d210006d65000072200000256c000064000000b5
:10d220000a0d0000637700005f6200007265000075
:10d23000616b00005f740000696d000065200000f4
:10d24000202500006c640000000a00000d6300004f
:10d25000775f000070650000726900006f64000075
:10d260002020000020200000202000002564000075
:10d27000000a00000d630000775f0000616300009a
:10d280007469000076650000202000002020000066
:10d290002020000025640000000a00000d2000008e
:10d2a0006b65000079650000725f00006d6f000023
:10d2b000646500002020000020200000256400009c
:10d2c000000a00000d4100004e54000020520000f2
:10d2d0004c59000020250000642c00002050000064
:10d2e0005454000020250000642c0000204200005f
:10d2f000554600004645000052200000256400000d
:10d300002c2000004357000020250000640000008e
:10d310000a0d00005365000072760000696300008a
:10d320006520000026200000636100006c69000099
:10d330006272000061740000696f00006e200000de
:10d340006d6f000064650000000a00000d440000dd
:10d3500049530000502000003d2000007061000093
:10d36000726100006d6500007465000072200000ad
:10d37000736500006c650000637400002c200000e1
:10d380004f50000045520000203d00002073000077
:10d39000617600006520000026200000657800000e
:10d3a0006974000000530000657400002052000002
:10d3b00065660000204f00007363000020460000f7
:10d3c00072650000710000004f73000063200000d0
:10d3d000256c000069200000487a00002020000031
:10d3e0000053000075700000706c00007920000090
:10d3f00020000000562000002000000043610000d3
:10d400006c2000006d7500006c740000203d000071
:10d41000202500006c690000202000002020000072
:10d420000042000065650000702000006c6500008f
:10d430006e2c0000203000003d4f000046460000ea
:10d44000200000004265000065700000203d0000e3
:10d4500020250000692000006d73000020200000de
:10d4600020200000004600006f720000776100007d
:10d4700072640000200000005246000020410000bd
:10d480006d7000002e2000002000000043610000ad
:10d490006c2000006d7500006c740000203d0000e1
:10d4a000202500006c6900002020000000430000df
:10d4b0005720000062720000656100006b200000d0
:10d4c00070650000726900006f64000020000000b9
:10d4d00025690000205500006e690000747300008b
:10d4e000202000002020000020200000202000003c
:10d4f000202000000050000075730000682000002c
:10d500004f50000045520000206c00006f6e00007c
:10d51000672000003d0000006661000063740000a9
:10d520006f720000792000006465000066610000f1
:10d53000756c000074730000004600006163000019
:10d54000746f0000727900002073000065740000a1
:10d5500075700000206f00006b0000000a0d0000d5
:10d5600046610000637400006f72000079200000c3
:10d570006465000066610000756c00007473000053
:10d580002072000065730000746f00007265000077
:10d5900064000000436100006c69000062720000da
:10d5a0002e2000005361000076650000640000003a
:10d5b0000a0d0000436100006c6900006272000007
:10d5c00061740000696f00006e2000007365000048
:10d5d00074740000696e000067730000207300001f
:10d5e0006176000065640000207400006f20000078
:10d5f00045450000505200004f4d00000000000063
:10d600000a0d000054520000415000003a20000072
:10d610004f730000636900006c610000746f0000cc
:10d620007220000045720000726f0000720a000054
:10d630000d0000004f530000434300004f4e000018
:10d640002030000078250000580a00000d0000007e
:10d650000a0d000054520000415000003a20000022
:10d6600041640000647200006573000073200000d4
:10d6700045720000726f0000720a00000d00000089
:10d68000573000002030000078250000580a0000c4
:10d690000d00000057310000203000007825000008
:10d6a000580a00000d000000573200002030000032
:10d6b00078250000580a00000d00000057330000d4
:10d6c0002030000078250000580a00000d000000fe
:10d6d000573400002030000078250000580a000070
:10d6e0000d000000573500002030000078250000b4
:10d6f000580a00000d0000005736000020300000de
:10d7000078250000580a00000d000000573700007f
:10d710002030000078250000580a00000d000000ad
:10d72000573800002030000078250000580a00001b
:10d730000d0000005739000020300000782500005f
:10d74000580a00000d000000573100003020000092
:10d7500030780000255800000a0d00000057000036
:10d76000313100002030000078250000580a000008
:10d770000d0000005731000032200000307800001a
:10d78000255800000a0d000000570000313300004a
:10d790002030000078250000580a00000d0000002d
:10d7a0005731000034200000307800002558000078
:10d7b0000a0d000000570000313500002030000045
:10d7c00078250000580a00000d0000000a0d000036
:10d7d00054520000415000003a20000053740000f1
:10d7e000616300006b20000045720000726f000052
:10d7f000720a00000d0000000a0d000054520000e3
:10d80000415000003a2000004d61000074680000a3
:10d8100020450000727200006f7200000a0d0000c7
:10d82000000a00000d5300007075000072690000ce
:10d830006f75000073200000496e000074650000e1
:10d8400072720000757000007420000045720000c4
:10d85000726f0000720a00000d000000202000001e
:10d860002020000045720000726f0000722000004e
:10d8700021200000202000002020000000000000e7
:10d880007f010000bf0000005f0000002f000000cb
:10d89000170000000b00000007000000030000005c
:10d8a0002000000000010000010200002003000031
:10d8b0000304000004020000060600000606000043
:10d8c000050700000707000020000000000000001e
:10d8d00000000000000000002d2e00002d2e000092
:10d8e0002d000000000000002e2d00002e2e000054
:10d8f0002d2e0000000000002e2d00002e2d000017
:10d900002e000000000000002e2e00002e2d000032
:10d910002e2e00002d00000020000000000000005e
:10d9200000000000000000002e2d00002e2e000040
:10d930002e000000000000002e2d00002d2d000004
:10d940002d2e0000000000002d2e00002d2d0000c7
:10d950002e000000000000002d2e00002d2d0000e4
:10d960002e2d0000000000002e2e00002e2d0000a5
:10d970002e2d0000000000002e2d00002e2d000096
:10d980002e000000000000002d2d00002e2e0000b3
:10d990002d2d0000000000002d2e00002e2e000076
:10d9a0002e2d0000000000002e2d00002e2d000066
:10d9b0002e2d0000000000002d2e00002e2d000056
:10d9c0002e000000000000002d2d00002d2d000075
:10d9d0002d000000000000002e2d00002d2d000065
:10d9e0002d000000000000002e2e00002d2d000054
:10d9f0002d000000000000002e2e00002e2d000043
:10da00002d000000000000002e2e00002e2e000031
:10da10002d000000000000002e2e00002e2e000021
:10da20002e000000000000002d2e00002e2e000011
:10da30002e000000000000002d2d00002e2e000002
:10da40002e000000000000002d2d00002d2e0000f3
:10da50002e000000000000002d2d00002d2d0000e4
:10da60002e000000000000002d2d00002d2e0000d3
:10da70002e2e0000000000002d2e00002d2e000094
:10da80002d2e00000000000020000000000000001b
:10da900000000000000000002d2e00002e2e0000cf
:10daa0002d00000000000000200000000000000029
:10dab00000000000000000002e2e00002d2d0000b0
:10dac0002e2e0000000000002e2d00002d2e000044
:10dad0002d2e0000000000002e2d00000000000090
:10dae00000000000000000002d2e00002e2e00007f
:10daf00000000000000000002d2e00002d2e000070
:10db000000000000000000002d2e00002e0000008c
:10db100000000000000000002e00000000000000d7
:10db200000000000000000002e2e00002d2e00003e
:10db300000000000000000002d2d00002e0000005d
:10db400000000000000000002e2e00002e2e00001d
:10db500000000000000000002e2e00000000000069
:10db600000000000000000002e2d00002d2d000000
:10db700000000000000000002d2e00002d0000001d
:10db800000000000000000002e2d00002e2e0000de
:10db900000000000000000002d2d0000000000002b
:10dba00000000000000000002d2e0000000000001a
:10dbb00000000000000000002d2d00002d000000de
:10dbc00000000000000000002e2d00002d2e00009f
:10dbd00000000000000000002d2d00002e2d000090
:10dbe00000000000000000002e2d00002e000000ac
:10dbf00000000000000000002e2e00002e0000009b
:10dc000000000000000000002d00000000000000e7
:10dc100000000000000000002e2e00002d0000007b
:10dc200000000000000000002e2e00002e2d00003d
:10dc300000000000000000002e2d00002d0000005c
:10dc400000000000000000002d2e00002e2d00001e
:10dc500000000000000000002d2e00002d2d00000f
:10dc600000000000000000002d2d00002e2e0000fe
:10dc70000000000000000000200000000000000084
:10dc80000000000000000000200000000000000074
:10dc90000000000000000000200000000000000064
:10dca0000000000000000000200000000000000054
:10dcb00000000000000000002e2e00002d2d0000ae
:10dcc0002e2d0000000000002e2d00002e2d000043
:10dcd00000000000000000002d2d00002d2e00008f
:10dce00000000000000000002e2d00002d2e00007e
:10dcf0002d000000000000002e2e00002d2d000041
:10dd000000000000000000003d4f000025690000f9
:10dd10000a0d0000003d0000462500002e360000e0
:10dd20006c6400000a0d0000003d0000543100004a
:10dd30000a0d0000003d0000543000000a0d0000f4
:10dd4000003d00004b250000690a00000d000000a6
:10dd50003d530000252e0000336400000a0d000032
:10dd6000003d000050250000690a00000d00000081
:10dd70003d580000256900000a0d0000003d00002c
:10dd800041250000690a00000d0000003d4300002d
:10dd9000256900000a0d0000003d00004d00000054
:10dda0000a0d0000003d000049490000004a000043
:10ddb000554d0000412d0000545800003530000042
:10ddc000300000004a5500004d4100002d54000075
:10ddd0005831000033360000005500004e4b000063
:10dde0004e4f0000574e0000002c00002053000052
:10ddf00057200000002c0000204400004154000087
:10de000045200000003d000049500000256400004e
:10de10000a0d0000003d0000495300002564000089
:10de20000a0d0000003d000049420000256400008a
:10de30000a0d0000003d0000494400002564000078
:10de40000a0d0000003d0000424300000a0d0000e2
:10de5000003d000042250000690a00000d0000009e
:020000040000fa
:10de60001e0c0000120000000200000000004a002a
:10de7000554d41002054580035303000205152009b
:10de80005600000000080000a6010000000000008d
:10de9000820b00003e00000000000000e20b0000ca
:10dea0002000000000000000a60900000c01000096
:10deb00000000000640c00000200000002000000ee
:10dec00001000000020c00001c0000000000000027
:10ded000300c00001200000000000000540c000094
:10dee0000a00000002000000000000000000000026
:10def0000000000000000000b20a000088000000de
:10df0000020000000100000000d80a00d90ad80071
:10df10000ad80a00d80ad8000ac80a00000000007f
:10df200000000000000000000000000000000000f1
:10df300000000000000000000002080001010000d5
:10df40000b010b00000b00000b000b00000bf0009e
:10df50000a000000000000000000000000000000b7
:10df600000000000000000000000000000000200af
:10df700008020200280b29000b280b00280b2800a0
:10df80000b280b00180b0000000000000000000030
:10df90000000000000000000000000000000000081
:10dfa00000000000b20ada000a020b0000000000c4
:10dfb000000000000000000000000000420c000013
:10dfc0001200000002000000202b2d002330000072
:10dfd0000100020000040000080010000000000022
:10dfe000a20c00000800000002000000686a6c003b
:10dff000747a4c00000000005e0c00000600000077
:10e00000020000000000000000000200660c00009a
:10e010000200000000000000c00b00002200000011
:10e02000020000003031320033343500363738001a
:10e03000396162006364650066003000313233008c
:10e0400034353600373839004142430044454600f4
:10e05000000000003a0b0000480000000200000031
:10e06000000000000000000024400000000000004c
:10e0700000005900400000000000000088c340007c
:10e08000000000000084d7009741000080e03700c6
:10e0900079c3410043176e0005b5b500b89346003b
:10e0a000f5f93f00e9034f00384d32001d30f9000b
:10e0b000487782005a3cbf00737fdd004f15750022
:10e0c000700c000032000000020000004e414e00c3
:10e0d000006e61006e0049004e460000696e6600e9
:10e0e00000303100323334003536370038396100c2
:10e0f00062636400656600003031320033343500fd
:10e10000363738003941420043444500460000009c
:10e11000680c000002000000020000000000000087
:10e12000aa0c000002000000020000003000000005
:10e130006a0c000002000000020000000000000065
:10e140006c0c000002000000020000000100000052
:10e150006e0c000002000000000000000000000043
:00000001FF
